:100000000C94AC070C94D4070C94D4070C94D4072C
:100010000C94D4070C94D4070C94D4070C94D407F4
:100020000C94D4070C94D4070C9472190C94E11915
:100030000C94D4070C94D4070C94D4070C94D407D4
:100040000C94D4070C94D4070C94D4070C94D407C4
:100050000C94D4070C94D4070C94D4070C94131C60
:100060000C94D4070C94D4070C94D4070C94D407A4
:100070000C94D4070C94D4070C94D4070C94D40794
:100080000C94D4070C94D4070C94D4070C94D40784
:100090000C94D4070C94D4070C94D4070C94D40774
:1000A0000C94D4070C94D4070C94D40744617900C1
:1000B00041636374004C6F616E00436170616369FA
:1000C0007479200047756E732000050512151F1501
:1000D0000905082466E766244120596573202042FB
:1000E000204E6F000042726F6F6B6C796E00436F31
:1000F0006E65792049736C616E64004D616E686154
:100100007474656E0043656E7472616C2050617228
:100110006B0047686574746F0042726F6E78000000
:100120004C7564657300537065656400576565645C
:100130000041636964004865726F696E6500436FD2
:100140006361696E65002000200003081F051F1F02
:10015000151B1F11111F110E1F15111F05011F1156
:100160001D1F041F001F0010101F1F041B1F101055
:100170001F061F1F011F1F111F1F05071F311F1FF4
:10018000051B17151D011F011F101F0F100F1F0C3E
:100190001F1B041B071C071915130C121E1F120C22
:1001A0001E12120C121F0C1A14041F052E2A1E1FD9
:1001B000021C001D00201D001F041A011F001E0448
:1001C0001E1E021E1E121E3E120C0C123E1E0206A7
:1001D00014120A020F121E101E0E100E1E081E1AF6
:1001E000041A2E281E1A12161F111F001F001D159B
:1001F0001711151F07041F17151D1F151D01011FBE
:100200001F151F17151F00170000100020100000F9
:10021000030004083E09093E3F25251A1E2121122C
:100220003F21211E3F2525213F0505011E21293A99
:100230003F04043F213F21001021211F3F040A31C8
:100240003F2020203F02023F3F02043F1E21211E8B
:100250003F0909061E21112E3F09093622252519BD
:10026000013F01011F20201F0F10201F3F10103FD2
:100270003B04043B03043807312D2321102A2A3C78
:100280003F2424181C2222141824243F1C2A2A2C20
:10029000047E05014C52523E3F040438243D2000A8
:1002A0004040443D3F081422213F20003E04043ECC
:1002B0003E04023C1C22221C7E22221C1C22227E86
:1002C0003E040204242A2A12021F22201E20201E7D
:1002D0000E10201E3E10103E360808364E50503E7E
:1002E000322A26221E29251E223F200032292926B5
:1002F0001221251A0C0A3F08172525191E25251835
:10030000013905031A25251A0629291E002F000088
:10031000002000004020000000030000000000005A
:10032000003E5B4F5B3E3E6B4F6B3E1C3E7C3E1C7B
:10033000183C7E3C181C577D571C1C5E7F5E1C00C1
:10034000183C1800FFE7C3E7FF0018241800FFE778
:10035000DBE7FF30483A060E2629792926407F053B
:100360000507407F05253F5A3CE73C5A7F3E1C1C51
:1003700008081C1C3E7F14227F22145F5F005F5F11
:1003800006097F017F006689956A606060606094FD
:10039000A2FFA29408047E040810207E2010080802
:1003A0002A1C08081C2A08081E101010100C1E0C0D
:1003B0001E0C30383E3830060E3E0E06000000009F
:1003C0000000005F00000007000700147F147F1486
:1003D000242A7F2A122313086462364956205000CB
:1003E00008070300001C2241000041221C002A1CB7
:1003F0007F1C2A08083E08080080703000080808A2
:100400000808000060600020100804023E514945C1
:100410003E00427F400072494949462141494D33DF
:100420001814127F1027454545393C4A4949314146
:10043000211109073649494936464949291E000014
:100440001400000040340000000814224114141469
:100450001414004122140802015909063E415D5955
:100460004E7C1211127C7F494949363E414141225E
:100470007F4141413E7F494949417F090909013E88
:10048000414151737F0808087F00417F41002040AF
:10049000413F017F081422417F404040407F021CC1
:1004A000027F7F0408107F3E4141413E7F090909D8
:1004B000063E4151215E7F091929462649494932A4
:1004C00003017F01033F4040403F1F2040201F3F6A
:1004D0004038403F631408146303047804036159EF
:1004E000494D43007F414141020408102000414131
:1004F000417F0402010204404040404000030708DD
:100500000020545478407F284444383844444428D8
:10051000384444287F385454541800087E0902187F
:10052000A4A49C787F0804047800447D4000204007
:10053000403D007F1028440000417F40007C04784B
:1005400004787C080404783844444438FC18242493
:100550001818242418FC7C08040408485454542413
:1005600004043F44243C4040207C1C2040201C3C90
:100570004030403C44281028444C9090907C446487
:10058000544C44000836410000007700000041361A
:10059000080002010204023C2623263C1EA1A161A0
:1005A000123A4040207A38545455592155557941D2
:1005B0002154547841215554784020545579400CA9
:1005C0001E5272123955555559395454545939558A
:1005D0005454580000457C410002457D42000145CD
:1005E0007C40F0292429F0F0282528F07C5455453A
:1005F000002054547C547C0A097F493249494932CD
:100600003248484832324A4848303A4141217A3AE1
:1006100042402078009DA0A07D39444444393D40AB
:1006200040403D3C24FF2424487E4943662B2FFC58
:100630002F2BFF0929F620C0887E09032054547906
:10064000410000447D413048484A32384040227AD7
:10065000007A0A0A727D0D19317D2629292F282654
:100660002929292630484D4020380808080808085C
:100670000808382F10C8ACBA2F102834FA00007BB5
:10068000000008142A142222142A140895002200BB
:1006900095AA005500AAAA55AA55AA000000FF0075
:1006A000101010FF00141414FF001010FF00FF10B2
:1006B00010F010F0141414FC001414F700FF0000E4
:1006C000FF00FF1414F404FC141417101F10101F63
:1006D000101F1414141F00101010F0000000001F51
:1006E000101010101F10101010F010000000FF105C
:1006F0001010101010101010FF10000000FF140058
:1007000000FF00FF00001F10170000FC04F4141489
:100710001710171414F404F40000FF00F714141455
:1007200014141414F700F7141414171410101F10D5
:100730001F141414F4141010F010F000001F101FF8
:100740000000001F14000000FC140000F010F01066
:1007500010FF10FF141414FF141010101F000000DD
:1007600000F010FFFFFFFFFFF0F0F0F0F0FFFFFFE1
:100770000000000000FFFF0F0F0F0F0F3844443838
:10078000447C2A2A3E147E02020606027E027E0273
:1007900063554941633844443C04407E201E200692
:1007A000027E020299A5E7A5991C2A492A1C4C72CF
:1007B00001724C304A4D4D303048784830BC625A56
:1007C000463D3E494949007E0101017E2A2A2A2AE6
:1007D0002A44445F444440514A444040444A5140C2
:1007E0000000FF0103E080FF000008086B6B083683
:1007F00012362436060F090F0600001818000000F4
:100800001010003040FF0101001F01011E00191DE2
:100810001712003C3C3C3C0000000000D5F08D1459
:10082000A1C881CFD9F1AF2000F0F89C8E878387D3
:100830008E9CF8F00000FEFF0303030303070EFC89
:10084000F80000FEFF0303030303070EFCF800009B
:10085000FFFF00000000000000FFFF0000FEFF831C
:1008600083838383C7EE7C380000F8FC0E07030304
:1008700003070EFCF800003F7FE0C08080C0E07FEF
:100880003FFFFF01010101010101FFFF0000FFFF28
:100890000C0C0C0C1C3E77E3C100007FFFC0C0C0F5
:1008A000C0C0E0703F1F00001F3F70E0C0C0C0E04C
:1008B000703F1F00007FFFC1C1C1C1C1E3773E1C73
:1008C00000001F3F70E0C0C0C0E0703F1F0000008C
:1008D000000001FFFF010000004861726461737352
:1008E000272063617263617373212100646F6C6CF4
:1008F000617273206F6E204F666669636572007463
:1009000068656D2120596F7520666F756E642000D3
:10091000596F75206B696C6C656420616C6C206F1D
:100920006600596F75206B696C6C6564206F6E652D
:10093000212100002020596F75206D697373656453
:1009400021212100006861766520746F2072756E28
:100950002100616E792067756E732120596F7500D3
:10096000596F7520646F6E27742068617665007416
:1009700068656D2100596F752063616E277420735F
:1009800068616B6500616E20616C6C657921210086
:10099000596F75206C6F7374207468656D20696E73
:1009A00000756E697473206F663A2000596F752068
:1009B000666F756E642000323030206275636B7331
:1009C0003F006D6F726520706F636B657473206696
:1009D0006F72007472656E6368636F61742077690B
:1009E00074680057696C6C20796F75206275792086
:1009F00061206E65770057696C6C20796F75207384
:100A00006D6F6B652069743F006C696B6520676F63
:100A10006F642073747566662121006865726520B5
:100A20007468617420736D656C6C730054686572D2
:100A300065277320736F6D65207765656400646F4B
:100A40006C6C6172733F007370656369616C2066E2
:100A50006F72203430300073617475726461792074
:100A60006E69676874002E3434206D61676E756D31
:100A700020666F72006261726574746120666F72C5
:100A80000034303020646F6C6C6172733F005769C2
:100A90006C6C20796F7520627579206100616674D5
:100AA000657220796F75210064657075746965736E
:100AB0002061726500206F662068697300616E6452
:100AC00020004F66666963657220486172646173D5
:100AD0007300696E2074686520737562776179218F
:100AE00000596F752077657265206D75676765645D
:100AF00000617265206F7574726167656F7573212F
:100B000021212100636F6B65206275737421205071
:100B100072696365730050696773206D6164652055
:100B20006120626967007072696365732121210029
:100B30006174206F7574726167656F75730062759B
:100B400079696E67206865726F696E6500416464DB
:100B50006963747320617265007261696421212187
:100B6000210066726F6D206C617374207765656B10
:100B70002773006368656170206865726F696E65D0
:100B80000050696773206172652073656C6C696ED3
:100B90006700626F74746F6D6564206F75742121D6
:100BA0002100576565642070726963657320686110
:100BB0007665006C756465732121210073656C6C2A
:100BC000696E6720636865617000526976616C20A8
:100BD0006465616C6572732061726500746F646135
:100BE000792100626F72726F776564206D6F6E6538
:100BF0007900596F7520616C72656164790021001C
:100C0000596F7520646F6E27742068617665206166
:100C10006E7900004F6F707321002100596F7520AD
:100C200063616E2774206166666F726400004F6FA7
:100C30007073210021006D6F72652000596F75205F
:100C400063616E277420636172727900004F6F7068
:100C5000732100596F7527726520646561642121D5
:100C6000006265656E206869742100596F7527768A
:100C700065006D69737365642121005468657900AE
:100C8000796F752121200054686579277265206687
:100C90006972696E672061740041204669676874F3
:100CA0002020422052756E004552524F5220004182
:100CB0006D7400536176696E677300596F75206FAC
:100CC000776500596F7520686176650057697468AB
:100CD00064726177204D6F6E6579004465706F7343
:100CE0006974204D6F6E657900426F72726F772064
:100CF0004D6F6E657900506179204C6F616E000018
:100D00000051747900507269636500436F737473A6
:100D100000596F7520686176650053656C6C200022
:100D20004275792000000075703F00646F63746F36
:100D30007220746F2073657720796F7500646F6C13
:100D40006C61727320666F7220610057696C6C2051
:100D5000796F7520706179203130303000596F75AE
:100D600072206865616C74683A20007374696C6CF9
:100D700020616674657220796F7521002070696743
:100D80007300546865726520617265200042656970
:100D90006E67206368617365642121005769746818
:100DA00064726177204D6F6E6579004465706F7372
:100DB0006974204D6F6E65790042616E6B00426F01
:100DC00072726F77204D6F6E657900526570617930
:100DD000204C6F616E004C6F616E20536861726BC6
:100DE000004A65742066726F6D200053656C6C203C
:100DF0004472756773004275792044727567730099
:100E00005472656E6368636F61740042616E6B005B
:100E10004C6F616E20536861726B004A65740054B8
:100E200072656E6368636F61740053656C6C204417
:100E30007275677300427579204472756773004854
:100E40006974207468652053747265657473212118
:100E50000076312E3000536C616E67696E27001E7C
:100E60001E0000C080000000000000000080780725
:100E7000067880000000000000000000C040000074
:100E800000033CC10204081020C000FF0000000065
:100E9000FF00C02010080404C23907000038509039
:100EA00090902324485060812608E70090E70826A8
:100EB0000160504826A19090905030000000000042
:100EC000010222322A2422100A080C081221242AA4
:100ED000320203000000000000080B0002020200C2
:100EE00000090400000102020000052400100105B1
:100EF00024010101042402060524060001070581DE
:100F00000310004009040100020A00000007050266
:100F10000240000007058302400000040309041298
:100F2000010002EF0201404123368000010102036B
:100F30000141726475696E6F204C4C4300417264CC
:100F400075696E6F204C656F6E6172646F0003058A
:100F50001F0E0400901CD12E11241FBECFEFDAE02B
:100F6000DEBFCDBF12E0A0E0B1E0E2E6FBE602C0EA
:100F700005900D92A236B107D9F727E0A2E6B2E0BC
:100F800001C01D92AC3AB207E1F717E0CBEAD7E017
:100F900004C02197FE010E94AC33CA3AD107C9F7B9
:100FA0000E94111D0C94A4350C940000E2EFF2E0B5
:100FB000A0E0B8E000800EBC8111012C1197A0FDCB
:100FC000FDCF0192B9F70DB40895480F592F511D67
:100FD0001416150684F5803891056CF597FF02C04C
:100FE00090E080E04138510514F040E850E0481BA3
:100FF000FB01E770FF2721E001C0220FEA95EAF725
:1010000077FF02C0695F7F4FFB0133E0F595E795FD
:101010003A95E1F7F695FE2FEE27F795E795E80F5D
:10102000F91FEE50FD4F415030F08191DF011197D3
:10103000822B8C93F8CF08956F927F928F929F921C
:10104000AF92BF92CF92DF92EF92FF920F931F93D6
:10105000CF93DF93DC01FA011491319654913196CC
:10106000C12FD0E0222309F1CC24C394D12C852FA9
:10107000877011F4D12CC12CE52EE694E694E69409
:10108000EC0CFD2CF11CEC9EC001ED9E900DFC9E25
:10109000900D1124033011F4880F991F289F7001BF
:1010A000299FF00C1124EE0DFF1D7D01EC0EFD1E9D
:1010B0001E141F040CF06BC0A038B1050CF067C003
:1010C000CB01850F911D181619060CF060C0603415
:1010D00071050CF05CC0309709F459C0362F377099
:1010E000CB0177FD079623E0959587952A95E1F743
:1010F000282F77FF04C0332311F02FEF280F662726
:1011000077276A1B7B0BB7FD02C070E060E090E8B8
:101110009A1B40E8E416F1040CF4912F961BE22E82
:10112000022E000CFF08DE2CD0942F3F0CF0D12CA7
:1011300041E0852F877009F440E0B52EB694B6944F
:10114000B6944B0DE40EF11C89E0E816F10414F09E
:1011500048E0421BB42EBD182D0D40E82403700159
:101160001124AE0DBF1DA60FB71F1D9D600D711D73
:101170001124AF01460F571FC32E032E000CDD08AC
:10118000033009F4C7C090F4023009F474C0DF9151
:10119000CF911F910F91FF90EF90DF90CF90BF9074
:1011A000AF909F908F907F906F9008950A3FA1F12C
:1011B000B20E0B3F61F72B1551F3BD016E507D4F01
:1011C00010E000E0091708F09FC0FA01E00FF11FDE
:1011D000E491F0E04F010C2C02C0880C991C0A9499
:1011E000E2F727FD06C0FB018081F82CF0948F21E7
:1011F0008083332361F0273054F47B01F0E8EF0E55
:10120000F11CA92CA094F70180818A2180830F5FB3
:101210001F4F6F5F7F4FD6CFB20E2B1509F4B7CF9C
:10122000BD016E507D4F10E000E0091708F066C068
:10123000FA01E00FF11FE491F0E04F010C2C02C025
:10124000880C991C0A94E2F727FD04C0FB018081F9
:1012500088298083332351F0273044F47B01F0E860
:10126000EF0EF11CF7018081892980830F5F1F4FEA
:101270006F5F7F4FDACF6FEF70E0032E02C0660F13
:10128000771F0A94E2F760957095972E8B2C820E4B
:10129000281509F47CCF8D010E501D4FF12CE12C47
:1012A000E91630F5FA01EE0DFF1DE491F0E03F0183
:1012B0000C2C02C0660C771C0A94E2F727FD05C0CF
:1012C000F8018081862386298083332359F02730D3
:1012D0004CF45801F0E8AF0EB11CF5018081892172
:1012E00087298083FFEFEF1AFF0A0F5F1F4FD8CFC8
:1012F0002F5F4C0F5D1FA058BF4FCACF2F5F4C0F01
:101300005D1FA058BF4F89CF2F5F4C0F5D1FA058A6
:10131000BF4F51CFE92EF12CFA01E60FF71FAE5067
:10132000BD4F60E870E06E197F09CE19DF098E01AC
:10133000000F111F41E050E07A01032E01C0EE0CB6
:101340000A94EAF7592F4B2D892E932ECF93DF93D2
:10135000ED01EF96EF962296A590C590992059F051
:10136000AE9C5001CE9C600127302CF4F880D094C4
:10137000FD20FB28F99222233AF0FC90C094FC2037
:10138000FA28FD920C94C50911965A9529F74A95A9
:1013900051F0582D23951124E00FF11DA60FB11D1A
:1013A000C60FD11DD9CFDF91CF911124F0CE0F936D
:1013B00002E020E00E941C080F9108952F923F92B6
:1013C0004F925F926F927F928F929F92AF92BF9255
:1013D000CF92DF92EF92FF920F931F93CF93DF9301
:1013E000CDB7DEB728970FB6F894DEBF0FBECDBFDE
:1013F0006F836A0119011C830B83FE82ED828111C8
:1014000028C005E010E029E030E03A832983B601E6
:101410000D2C000C880B990B0E9410304B015C01C5
:101420005F8151111DC0E0E6F7E090E080E0188692
:101430001F828C159D050CF02BC1248135814F81B5
:1014400058854217530714F438872F830196369630
:10145000F0CF04E010E048E050E05A834983D7CF52
:1014600020E030E040E05FE30E946F304B015C0120
:1014700020E030E0A9010E944A3320E030E040E063
:101480005FE387FD30C0C501B4010E94DE310E94D8
:10149000BC3278876F83A6018F819885481B590BD2
:1014A000E0E6F7E090E080E0B12CA12C2F813885B8
:1014B00082179307ECF086E0829FF001839FF00D86
:1014C0001124E05AF84F90E080E0D12CC12C841711
:1014D0009507BCF424813581C216D3060CF469014A
:1014E00001963696F4CFC501B4010E94DD31CFCF0D
:1014F00024813581A216B3060CF459010196369663
:10150000D5CFB801110F880B990B0E9410302B0119
:101510003C01B5016C0D7D1D072E000C880B990B4D
:101520000E94103020E030E040EE5FE30E94DE31A8
:101530006B017C0120E030E040E05FE3C301B201D9
:101540000E946F309B01AC01C701B6010E946F3051
:101550006B017C0120E030E0A9010E944A3320E0C9
:1015600030E040E05FE387FD89C0C701B6010E941B
:10157000DE310E94BC3202E410E0061B170BF101C1
:1015800011830083B501BB0C880B990B0E941030AE
:1015900020E030E040EE5FE30E94DE31A3019201E3
:1015A0000E946F304B015C0120E030E0A9010E94F5
:1015B0004A3320E030E040E05FE387FD64C0C501CE
:1015C000B4010E94DE310E94BC32600F711FEB81BA
:1015D000FC817183608329813A81B901330F880BC3
:1015E000990B0E94103020E030E040E05FE30E9461
:1015F0006F306B017C014F815885BA01550F880B04
:10160000990B0E9410309B01AC01C701B6010E94EA
:101610006F306B017C0120E030E0A9010E944A3369
:1016200020E030E040E05FE387FD85C0C701B60100
:101630000E94DE310E94BC322AE230E0C901861BE2
:10164000970BED81FE819183808328960FB6F894E5
:10165000DEBF0FBECDBFDF91CF911F910F91FF90E5
:10166000EF90DF90CF90BF90AF909F908F907F9042
:101670006F905F904F903F902F900895C701B601F3
:101680000E94DD3176CFC501B4010E94DD319BCFD0
:10169000B801110F880B990B0E94103020E030E048
:1016A00040E05FE30E946F302B013C01EF81F88541
:1016B000BF01FF0F880B990B0E9410309B01AC01FA
:1016C000C301B2010E946F302B013C0120E030E0E9
:1016D000A9010E944A3320E030E040E05FE387FD4B
:1016E00025C0C301B2010E94DE310E94BC3222E457
:1016F00030E0C901861B970BF101918380838FEF46
:101700009FEFEB81FC819183808329813A81B9012C
:10171000330F880B990B0E94103020E030E040E03E
:101720005FE30E946F30A501940171CFC301B20144
:101730000E94DD31DACFC701B6010E94DD317ACFD8
:10174000FC018091F102882311F13FB7F89482E007
:101750008093E9002091F200822F90E0181619067C
:1017600014F481E090E0882339F0289844E640930F
:10177000F0024091F1004083222339F02091F200E1
:10178000211103C02BE62093E8003FBF08958FEF9F
:101790009FEF08952FB7F89483E08093E90090912C
:1017A000E800892F807295FF04C09091F20080E4D8
:1017B000891B2FBF08958091E80281110DC082E03E
:1017C0008093E40284E08093E5021092E702109295
:1017D000E60281E08093E80284EE92E00895CF93E0
:1017E000DF931F92CDB7DEB76983DC01ED91FC91E9
:1017F0000280F381E02D41E050E0BE016F5F7F4F3A
:1018000009950F90DF91CF91089583E08093E900CF
:101810008091F200882319F08AE38093E80008950C
:101820000E94CA0B90E00895CF93DF931F92CDB72B
:10183000DEB7FC018485958597FD08C02FEF3FEF4B
:10184000358724870F90DF91CF910895CE010196BF
:101850000E94A00B019719F4898190E0F3CF8FEFDC
:101860009FEFF0CF0F931F93CF93DF931F92CDB7CE
:10187000DEB78C01FC018485958597FF0BC0CE01F6
:1018800001960E94A00B019771F4898190E0F80104
:1018900095878487F801848595850F90DF91CF9196
:1018A0001F910F9108958FEF9FEFF1CFFC01848579
:1018B000958597FD0BC09FB7F89482E08093E9006F
:1018C0008091F2009FBF90E0019608959FB7F89431
:1018D00082E08093E9008091F2009FBF90E008953C
:1018E0004091DE025091DF022091DC023091DD0256
:1018F00042175307B4F49091E8009570E1F390918A
:10190000E80092FD19C08093F1008091DE02909171
:10191000DF0201968F739927892B19F48EEF80933C
:10192000E8008091DE029091DF0201969093DF0241
:101930008093DE0281E0089580E00895DF92EF92C7
:10194000FF920F931F93CF93DF93D82E8A01EB0161
:101950007B01E40EF51ECE15DF0559F0D7FE12C04F
:10196000FE0184910E94700C21968111F4CF0FEF3B
:101970001FEFC801DF91CF911F910F91FF90EF9062
:10198000DF9008958881EECF0F931F93CF93DF935D
:101990001F92CDB7DEB782E0898342E450E069ED63
:1019A0007EE080E80E949E0C0E94DB0BDC01129618
:1019B0000D911C910115110589F0D801ED91FC9153
:1019C0000280F381E02DBE016F5F7F4FC801099552
:1019D00097FD04C0F80100851185ECCF89810F9037
:1019E000DF91CF911F910F910895615030F02091B8
:1019F000F100FC0120830196F8CF289884E68093BB
:101A0000F00208953FB7F8948091D8029091D902DE
:101A1000A091DA02B091DB0226B5A89B05C02F3F4A
:101A200019F00196A11DB11D3FBFBA2FA92F982F04
:101A30008827BC01CD01620F711D811D911D42E0FF
:101A4000660F771F881F991F4A95D1F708958F92C7
:101A50009F92AF92BF92CF92DF92EF92FF926B0173
:101A60007C010E94020D4B015C01C114D104E10410
:101A7000F104B9F00E94020D681979098A099B09DD
:101A8000683E73408105910580F321E0C21AD108B8
:101A9000E108F10888EE880E83E0981EA11CB11CB5
:101AA000E4CFFF90EF90DF90CF90BF90AF909F90EA
:101AB0008F9008958F929F92AF92BF92CF92DF92B4
:101AC000EF92FF920F931F93CF93DF936C017B01F3
:101AD0008A0180910C01882309F45CC08091F10295
:101AE000882309F457C08091E30280FF05C08091EC
:101AF000E00082608093E000E801B12C8AEFA82E1C
:101B000093E0892E2AE3922E209711F4BB20D9F17D
:101B10000E94CA0B81110AC0AA94AA20D9F161E0DF
:101B200070E080E090E00E94270DEECF8C171D063C
:101B300011F00CF08C2F9FB7F8948092E90020915F
:101B4000E80025FD02C09FBFDFCF282F30E0C21B79
:101B5000D30BF701815020F041914093F100FACF6F
:101B6000E20EF31EBB2021F09092E800B12CEBCFE7
:101B70008091E80085FDE7CF9092E800BB24B39404
:101B8000209709F3F3CF5D9884E68093E202101664
:101B900011063CF081E090E0F6019383828310E02F
:101BA00000E0C801DF91CF911F910F91FF90EF905E
:101BB000DF90CF90BF90AF909F908F900895089541
:101BC000DB0114964D915C9115976D917C91DC0130
:101BD000ED91FC910280F381E02D09942F923F92C8
:101BE0004F925F926F927F928F929F92AF92BF922D
:101BF000CF92DF92EF92FF920F931F93CF93DF93D9
:101C000000D000D000D0CDB7DEB7782E662E5A01B6
:101C100028E0422E512C811103C099E0492E512C0D
:101C2000CE0101967C018E010D5F1F4F9E012B5F3F
:101C30003F4FA501662D872D0E94DE09B5010B2CB3
:101C4000000C880B990B0E94103020E030E040E03F
:101C50005FE30E946F306B017C0120E030E0A9015E
:101C60000E944A3320E030E040E05FE387FD24C07B
:101C7000C701B6010E94DE310E94BC328B0180E6B2
:101C8000C82E87E0D82E049D1001059D300C149DB0
:101C9000300C1124F12CE12C912C812C8A149B0402
:101CA000B4F589819A81662019F0801691064CF46A
:101CB0002D818E0D9F1D0BC0C701B6010E94DD3125
:101CC000DBCF2B81A70142195309840F951F772081
:101CD000A1F0209395072093940780939607B6016F
:101CE00080E997E00E94E00D9FEF891A990A86E04B
:101CF000C80ED11CE40CF51CD1CF20939F07209374
:101D00009E078093A007B6018AE997E0EBCF26965D
:101D10000FB6F894DEBF0FBECDBFDF91CF911F91FC
:101D20000F91FF90EF90DF90CF90BF90AF909F907A
:101D30008F907F906F905F904F903F902F9008957D
:101D4000EF92FF920F931F93CF93DF938C017B0150
:101D5000D0E0C0E0F701EC0FFD1F6491662361F055
:101D6000D801ED91FC910190F081E02DC801099519
:101D7000892B11F02196EECFCE01DF91CF911F91EB
:101D80000F91FF90EF900895AF92BF92CF92DF92A4
:101D9000EF92FF920F931F93CF93DF936C017B0120
:101DA0008B01040F151FEB015E01AE18BF08C017B1
:101DB000D10759F06991D601ED91FC910190F08124
:101DC000E02DC6010995892B79F7C501DF91CF91E7
:101DD0001F910F91FF90EF90DF90CF90BF90AF9049
:101DE00008952D9A0895BC0190E080E00C94270D91
:101DF0008FB18095807F669B88601C9B846008956E
:101E000081EC80937C0085B1806F85B984B1877E39
:101E100084B984B1876E84B95E9A5F988AB1806D07
:101E20008AB9769A6E9881B3806F81BB899880B3A6
:101E30008D7080BB80E58CBD81E08DBD85E090E03C
:101E40000E94F30E5F9A85E090E00E94F30E5E9888
:101E50005C98ECE1F8E084918EBD00000DB407FEC3
:101E6000FDCF319688E0E932F807A9F75C9A81E85E
:101E7000809364008091650081608093650008957F
:101E800090916A02982329F490916B02982381E043
:101E900009F480E00895CF93C82F0E94F80E982F80
:101EA0009C2381E09C1380E0CF91089580E00C9406
:101EB000D60780389105B8F460347105A0F420E1AC
:101EC00091E061FD94E060FD990F62FD9295687F5D
:101ED000269FD0011124A80FAE50BD4F8C9140FF1A
:101EE00003C0892B8C93089590958923FBCF2F9263
:101EF0003F924F925F926F927F928F929F92AF929A
:101F0000BF92CF92DF92EF92FF920F931F93CF93E6
:101F1000DF937C016B0188248394912CD0E0C0E096
:101F200005E010E096EF692E77247A942CEFA22E2C
:101F3000BB24BA94842F8470582E842F8270482E2C
:101F4000842F8870382E4170242E219682E0880ECE
:101F5000911CA80CB91C552091F041E0B8016C0D02
:101F60007D1DC7018C0F9D1F0E94590F41E0B601D6
:101F70006C0F7D1FC8018E0D9F1D0E94590F4420BC
:101F800091F041E0B601601B710BC7018C0F9D1FE2
:101F90000E94590F41E0B6016C1B7D0BC8018E0DEC
:101FA0009F1D0E94590F332091F041E0B6016C0F44
:101FB0007D1FC701801B910B0E94590F41E0B801A2
:101FC0006C0D7D1DC7018C1B9D0B0E94590F22209B
:101FD00091F041E0B6016C1B7D0BC701801B910B9A
:101FE0000E94590F41E0B601601B710BC7018C1BA9
:101FF0009D0B0E94590FC017D10754F4B7FCA5CF11
:102000000150110982E0680E711CA60CB71C9DCF0F
:10201000DF91CF911F910F91FF90EF90DF90CF90C4
:10202000BF90AF909F908F907F906F905F904F90F8
:102030003F902F9008952F923F924F925F926F9210
:102040007F928F929F92AF92BF92CF92DF92EF9248
:10205000FF920F931F93CF93DF93EC0141E06FE367
:1020600070E00E94590F41E065E370E0CE010E94EC
:10207000590F41E06AE370E0CE0105960E94590FC6
:1020800041E06AE370E0CE0105970E94590F2224D7
:102090002394312CF12CE12C05E010E036EF432E97
:1020A00055245A944CEFC42EDD24DA948FEFE81AAD
:1020B000F80A82E0280E311CC20CD31C47018C0E9A
:1020C0009D1E41E058018AE3A80EB11CB501C40170
:1020D0000E94590F3E016E187F0841E0B501C3010F
:1020E0000E94590F41E08AE3A82EB12CA01AB10A30
:1020F000B501C4010E94590F41E0B501C3010E941E
:10210000590F47018AE3880E911C41E0B4015E013A
:10211000A00EB11EC5010E94590F41E0B4013E015D
:10212000601A710AC3010E94590F9AE3892E912CFB
:102130008E189F0841E0B401C5010E94590F41E08B
:10214000B401C3010E94590FE016F1069CF0DF9123
:10215000CF911F910F91FF90EF90DF90CF90BF90A4
:10216000AF909F908F907F906F905F904F903F9037
:102170002F900895D7FC9ACF0150110982E0480EA4
:10218000511CC40CD51C92CF8F929F92AF92BF92DC
:10219000CF92DF92EF92FF920F931F93CF93DF9333
:1021A0006D3089F0C0906802D09069026A30D1F435
:1021B000109267021092660288E0C80ED11CD0927D
:1021C0006902C092680281E090E0DF91CF911F9197
:1021D0000F91FF90EF90DF90CF90BF90AF909F90C6
:1021E0008F9008950091660210916702E5E06E9F5E
:1021F000E0011124C45EDC4F4801F12CF5E0E12C34
:10220000FF1629F0CE010196FE01E490EC01B12CFD
:10221000A12C4E2D4170B6016A0D7B1DC4010E9498
:10222000590FE694FFEFAF1ABF0A88E0A816B10471
:1022300081F7F394EFEF8E1A9E0AF6E0FF12DECFDD
:102240000A5F1F4F1093670200936602BCCFDF92B4
:10225000EF92FF920F931F93CF93DF937C01D22EC7
:102260008B01040F111DEB0177FF02C0D0E0C0E02D
:10227000C8010134110514F080E490E0C817D907B3
:102280003CF44D2DBE01C7010E94590F2196F0CF9D
:10229000DF91CF911F910F91FF90EF90DF90089504
:1022A0002F923F924F925F926F927F928F929F9266
:1022B000AF92BF92CF92DF92EF92FF920F931F9354
:1022C000CF93DF9300D000D000D0CDB7DEB76C0144
:1022D000762E542E4901602E98E0A92EB12C611162
:1022E00003C089E0A82EB12CCE0101967C018E019D
:1022F0000D5F1F4F9E012B5F3F4FA401652D872D62
:102300000E94DE0909811A81552011F1B401990C4E
:10231000880B990B0E94103020E030E040E05FE332
:102320000E946F301B012C0120E030E0A9010E94C7
:102330004A3320E030E040E05FE387FD0CC0C2019B
:10234000B1010E94DE310E94BC32C616D70644F4A9
:102350008D809E8009C0C201B1010E94DD31F3CFA2
:102360008B809C80C61AD70ACA9CB001CB9C700D8A
:10237000DA9C700D1124060F171FC4010497662004
:10238000B1F061E070E0711002C062E070E0060F31
:10239000171F6C01C6012FEFC21AD20AC814D90444
:1023A00091F020E045E0B8010E942711F3CF61E0F1
:1023B00070E0711002C062E070E0600F711F4EE4C7
:1023C0005FE00E94D70926960FB6F894DEBF0FBED5
:1023D000CDBFDF91CF911F910F91FF90EF90DF90D4
:1023E000CF90BF90AF909F908F907F906F905F90B5
:1023F0004F903F902F9008950F93CF93DF93EC0170
:102400009E816A3059F48D818C836985960F9E83F5
:1024100081E090E0DF91CF910F910895262F61E048
:10242000690F2A3398F4203378F5273249F140F4C4
:10243000213261F198859C5F8C81890F8C83E8CF74
:102440002C3231F12E32B1F72FE309C0213490F351
:102450002B35C0F08FE9820F27548A3158F7062EAA
:10246000000C770B8C81082E000C990B3F810AEF32
:10247000313009F00BEF42E152E00E941C08DACF44
:1024800021E4EDCF2154EBCF2C5FE9CF2EE3E7CF52
:1024900020E4E5CF0F93CF93DF93EC019E816A3068
:1024A00059F48D818C836985960F9E8381E090E03D
:1024B000DF91CF910F910895262F61E0690F2A33A4
:1024C00098F4203378F5273249F140F4213261F154
:1024D00098859D5F8C81890F8C83E8CF2C3231F1F8
:1024E0002E32B1F72FE309C0213490F32B35C0F021
:1024F0008FE9820F27548A3158F7062E000C770B8C
:102500008C81082E000C990B3F810AEF313009F0C5
:102510000BEF4AE451E00E941C08DACF21E4EDCF32
:102520002154EBCF2C5FE9CF2EE3E7CF20E4E5CFBA
:10253000EEEAF2E026EC32E090E080E04191519149
:1025400061917191840F951F2E173F07B9F7409144
:102550007D0250917E0265E0649F9001659F300D81
:102560001124280F391F80917B0290917C02821BDD
:10257000930B0895CF93C82F84E00E94400F8111E0
:1025800007C0CC2381F088E00E94400F882359F0D7
:102590001092D20280918D0290918E029093CF0280
:1025A0008093CE0281E0CF910895E0E9F7E08AE4DC
:1025B0008583848387E3868368ED70E0CF010E9482
:1025C000A00E8BE490E00E941B1087E690E00C9434
:1025D0001B10CF92DF92EF92FF920F931F93CF9336
:1025E000DF9346E770E060E085E090E00E94E50759
:1025F00046E76FE370E085E090E00E94E50721E0A8
:1026000046E365E070E090E080E00E94271121E061
:1026100046E365E070E08FE790E00E94271141E01B
:1026200065E070E085E090E00E94770F42E065E0B1
:1026300070E08AE790E00E94770F44E06AE370E080
:102640008AE790E00E94770F48E06AE370E085E057
:1026500090E00E94770F80918F02C2E4D7E0811151
:1026600022C00AE010E0F12CE12C8AE0C82ED12C27
:102670008091900290919102E816F90684F58FEF0F
:10268000E81AF80AD0926702C092660210936902B3
:1026900000936802BE0184EA97E00E94E00D065FA5
:1026A0001F4F2696E5CF1AE0F12CE12C0AE080912D
:1026B000900290919102E816F9068CF400939F071E
:1026C00000939E071093A007BE018AE997E00E943D
:1026D000E00D8FEFE81AF80A175F2696E8CFDF9132
:1026E000CF911F910F91FF90EF90DF90CF900895C1
:1026F000BC01EAE9F7E096E0958394838CE0868359
:10270000CF010C94E00D90E080E008958F929F92AD
:10271000AF92BF92EF92FF920F931F93CF93DF93ED
:10272000CDB7DEB7A1970FB6F894DEBF0FBECDBF11
:102730007C01FA01CB0119A2223008F42AE08E01B3
:102740000F5D1F4F822E912CB12CA12CBF01A50132
:1027500094010E94AC31F901CA016A3074F5605DE0
:10276000D8016E938D01232B242B252B79F790E034
:1027700080E0109789F0FD0101900020E9F7319782
:10278000AF014A1B5B0BD701ED91FC910280F381F5
:10279000E02DB801C7010995A1960FB6F894DEBFE8
:1027A0000FBECDBFDF91CF911F910F91FF90EF90A2
:1027B000BF90AF909F908F900895695CD1CFCF92DA
:1027C000DF92EF92FF920F931F93CF93DF9377FFE8
:1027D00021C06A017B01EC01E881F9810190F0815F
:1027E000E02D6DE209958C0144275527BA014C195B
:1027F0005D096E097F092AE0CE010E948613800FD1
:10280000911FDF91CF911F910F91FF90EF90DF907B
:10281000CF9008952AE0DF91CF911F910F91FF9003
:10282000EF90DF90CF900C948613CF93DF93CFE19E
:10283000D0E020E04AE067E170E0CE010E9427117D
:102840002196CF36D105A9F783E280939F07809325
:102850009E0788E18093A00740917702509178020B
:102860006091790270917A028AE997E0DF91CF91C5
:102870000C94DF13BC01EAE9F7E09AE095839483B6
:1028800088E18683CF010E94E00D48E566E170E0B3
:102890008EE190E00E94E50748E561E270E08EE19C
:1028A00090E00E94E50721E04CE066E170E08EE1F7
:1028B00090E00E94271121E04CE066E170E085E79E
:1028C00090E00E9427110E94151441ED50E068E14C
:1028D00070E08FE690E00C94D709CF92DF92EF92F0
:1028E000FF920F931F93CF93C82F8B0169017A0139
:1028F0006E5F7F4F4AEC50E00E94D709CA5FEAE959
:10290000F7E0C583C4830683B701A601CF01CF9149
:102910001F910F91FF90EF90DF90CF900C94DF13F9
:10292000CF93DF938091CE029091CF02419702978F
:1029300068F5C8E2D0E020E047E065E270E0CE0153
:102940000E9427112196CF37D105A9F7E0918B027C
:10295000F0918C02EE0FFF1FEE0FFF1FEA56FD4FA6
:102960002081318142815381609177027091780298
:102970008091790290917A020E949C339B01AC0174
:1029800065E270E088E290E00E946D14DF91CF91E3
:102990000C941514CF93DF93EC01888199810097F3
:1029A00011F00E944E34198218821D821C821B82F3
:1029B0001A82DF91CF910895FC0180819181009767
:1029C00011F00C944E340895CF93C82F8091CC020F
:1029D0009091CD0201969093CD028093CC021092FB
:1029E00076020E94402F21EE3EE240E050E00E943D
:1029F00043316058714C8F4F9F4F60939602709394
:102A0000970280939802909399020E94402F29E5A3
:102A10003BE140E050E00E94433168577C4E8F4FCD
:102A20009F4F60939A0270939B0280939C029093B5
:102A30009D020E94402F23E230E040E050E00E94DF
:102A400043319B01AC01265F3F4F4F4F5F4FA4E6E0
:102A5000B0E00E94623160939E0270939F02809367
:102A6000A0029093A1020E94402F2BE230E040E0B0
:102A700050E00E9443319B01AC012F5D3F4F4F4F0F
:102A80005F4FAAE0B0E00E9462316093A2027093AF
:102A9000A3028093A4029093A5020E94402F20E1FC
:102AA00030E040E050E00E9443319B01AC01295FDF
:102AB0003F4F4F4F5F4FAAE0B0E00E9462316093FA
:102AC000A6027093A7028093A8029093A9020E9485
:102AD000402F25E030E040E050E00E9443319B0170
:102AE000AC012F5F3F4F4F4F5F4FAAE0B0E00E9415
:102AF00062316093AA027093AB028093AC02909310
:102B0000AD02CC23C1F16091830270918402809167
:102B10008502909186020E9410302DEC3CEC4CE82E
:102B20005FE30E946F300E94F2320E94BC326093D9
:102B30008302709384028093850290938602609151
:102B40007F027091800280918102909182020E94A6
:102B5000103024E13EEA47E85FE30E946F300E94B4
:102B6000F2320E94BC3260937F02709380028093A5
:102B70008102909382021092D202CF9108950C9418
:102B80002D310F931F93CF93DF938C01EB01FC0149
:102B9000808191810097E1F06881798161157105EB
:102BA000A9F0428153812C813D814217530770F077
:102BB0000E949D358C819D81F801958384831D82BF
:102BC0001C82DF91CF911F910F9108950E944E3486
:102BD00088819981F801918380838A819B81938385
:102BE00082838C819D8195838483198218821B82C4
:102BF0001A82E5CF0F931F93CF93DF93EC01888167
:102C00009981009759F02A813B812617370730F0C8
:102C100081E0DF91CF911F910F9108958B016F5F3C
:102C20007F4F0E94D734009759F0998388831B8384
:102C30000A832C813D81232B59F7FC011082E8CFB8
:102C400080E0E7CFEF92FF920F931F93CF93DF9334
:102C5000EC017B01CB010E949F2F0097A9F00C8112
:102C60001D81080F191FB801CE010E94FA15882393
:102C700061F0288139818C819D81B701820F931F7A
:102C80000E94982F1D830C8381E0DF91CF911F91CB
:102C90000F91FF90EF900895EF92FF920F931F9383
:102CA000CF93DF93FB01E080F180E114F10441F464
:102CB00080E0DF91CF911F910F91FF90EF900895E9
:102CC0000481158101151105B1F0EC018C819D8104
:102CD000080F191FB801CE010E94FA15882341F38D
:102CE000288139818C819D81B701820F931F0E94B9
:102CF0009D351D830C8381E0DCCFEF92FF920F9313
:102D00001F93CF93DF93EC018B016115710551F097
:102D1000CB010E949F2F7C01BC01CE010E94FA15BD
:102D200081110BC0CE010E94CA14CE01DF91CF9158
:102D30001F910F91FF90EF900895FD82EC82B801F2
:102D4000888199810E94982FF0CFFC011182108216
:102D500013821282158214820C947D16CF93DF9316
:102D6000EC016230710501F148F46115710581F0E3
:102D700061307105B1F06FE171E00CC06430710534
:102D8000C9F0A8F065307105B1F760E271E002C0EA
:102D90006EE371E0CE010E94A516CE01DF91CF91C6
:102DA000089566E371E0F6CF61E371E0F3CF6CE282
:102DB00071E0F0CF66E271E0EDCFCF93DF93EC01ED
:102DC0006230710501F148F46115710581F06130DF
:102DD0007105B1F064EE70E00CC064307105C9F0AB
:102DE000A8F065307105B1F765EE70E002C069E1E9
:102DF00071E0CE010E94A516CE01DF91CF9108951A
:102E000062E171E0F6CF65E071E0F3CF6BEF70E067
:102E1000F0CF6EEE70E0EDCFEF92FF920F931F9325
:102E2000CF93DF93EC017B018A01BA010E94FA156E
:102E300081110BC0CE010E94CA14CE01DF91CF9147
:102E40001F910F91FF90EF9008951D830C83B701A0
:102E5000888199810E949D35F0CFFB01019000206F
:102E6000E9F73197AF01461B570B0C940C170F93E2
:102E70001F93CF93DF93CDB7DEB762970FB6F89469
:102E8000DEBF0FBECDBF8C01CB01F80111821082D5
:102E900013821282158214824AE0BE016F5F7F4F57
:102EA0000E94A82FBE016F5F7F4FC8010E942D179F
:102EB00062960FB6F894DEBF0FBECDBFDF91CF9103
:102EC0001F910F9108950F931F93CF93DF93CDB769
:102ED000DEB7A2970FB6F894DEBF0FBECDBF8C0150
:102EE000CB01BA01F801118210821382128215827D
:102EF00014822AE0AE014F5F5F4F0E94B32FBE01E4
:102F00006F5F7F4FC8010E942D17A2960FB6F894ED
:102F1000DEBF0FBECDBFDF91CF911F910F910895FE
:102F20002F923F924F925F926F927F928F929F92D9
:102F3000AF92BF92CF92DF92EF92FF920F931F93C7
:102F4000CF93DF93CDB7DEB762970FB6F894DEBFAD
:102F50000FBECDBF2C019E012F5F3F4F49013901AC
:102F60001C01D12CC12C10E000E0B12CA12CF101EE
:102F700041915191619171911F01CE010D960E9475
:102F80006317E988FA88CE010D960E94DC14B60119
:102F9000CE010D960E94AE1689899A89E80EF91E17
:102FA000FFEFEF1AFF0AF301E192F1923F01CE0128
:102FB0000D960E94DC14F3E0CF16D1040CF03FC054
:102FC000AE14BF040CF457012FEFC21AD20A36E038
:102FD000C316D10461F680E6C82E87E0D82EF12C06
:102FE000E12C150183E0E816F1040CF01801B7019B
:102FF000CE010D960E94AE16BE01635F7F4FC601E3
:103000000E94C115CE010D960E94DC1468E471E0A7
:10301000C6010E942216712C612CF40180819181DD
:103020009101281B390B6216730674F466E471E093
:10303000C6010E9422163FEF631A730AEECF0E15E7
:103040001F0514F68701C0CFF201419151916191A2
:1030500071912F01CE010D960E946317BE01635F2F
:103060007F4FC6010E944C16CE010D960E94DC14C3
:10307000FFEFEF1AFF0A26E0C20ED11C32E0830EEA
:10308000911C86E0E816F10409F0ABCFF092CB0278
:10309000E092CA0281E08093C8020A0D1B1D07312D
:1030A00011050CF480E08093C90262960FB6F89483
:1030B000DEBF0FBECDBFDF91CF911F910F91FF906B
:1030C000EF90DF90CF90BF90AF909F908F907F90C8
:1030D0006F905F904F903F902F900895EF92FF92E6
:1030E0000F931F93CF93DF9300D000D000D0CDB7C4
:1030F000DEB78091CE029091CF02099709F05EC0B1
:103100000E9498128C01BC01CE0101960E943717D3
:10311000ED80FE80CE0101960E94DC1481E0809358
:103120009507809394071092960764EC70E080E90D
:1031300097E00E94A00E40917D0250917E02052EE4
:10314000000C660B770B80E997E00E94DF1387E1A4
:1031500090E08E199F09880F991F880F991F8093FF
:10316000950780939407109296076AEB70E080E9C8
:1031700097E00E94A00EA801110F660B770B80E963
:1031800097E00E94DF1310E000E021E041E068E0FA
:1031900070E0C8010E9427110F5F1F4F0038110512
:1031A000A1F726960FB6F894DEBF0FBECDBFDF9114
:1031B000CF911F910F91FF90EF900895409187025A
:1031C000509188026091890270918A02CE01019625
:1031D0000E946317ED80FE80CE0101960E94DC14F0
:1031E00000E210E00E191F09000F111F000F111F40
:1031F0008091CE029091CF029C012550310922305E
:10320000310508F052C021E02093950720939407E0
:103210001092960760EB70E0059711F465EB70E093
:1032200080E997E00E94A00E4AEC50E061E070E077
:1032300083E190E00E94D70989E18093950780930C
:103240009407109296078091CE029091CF02059735
:1032500019F540918302509184026091850270912A
:10326000860280E997E00E94DF134AEC50E061E0BB
:1032700070E0C80106970E94D70900939507009354
:1032800094071092960740918702509188026091AE
:10329000890270918A0273CF40917F02509180021F
:1032A0006091810270918202DCCF81E0809395076A
:1032B00080939407109296076CEA70E080E997E09B
:1032C0000E94A00E8EE08093950780939407109241
:1032D00096074091CC025091CD02052E000C660B52
:1032E000770BBFCF1F920F920FB60F9211248F93BF
:1032F0009F938091E1009091E100937F9093E10092
:1033000083FF0FC01092E90091E09093EB001092C0
:10331000EC0092E39093ED001092F10298E090930C
:10332000F00082FF22C093E09093E9009091F200B8
:10333000992319F09AE39093E8009091E20299237F
:1033400041F09091E20291509093E202911101C0FC
:103350005D9A9091F002992341F09091F002915082
:103360009093F002911101C0289A84FF18C08091B7
:10337000E2008E7E81608093E2008091E1008F7E8A
:103380008093E1008091E3028E7E80618093E3026E
:103390009F918F910F900FBE0F901F90189580FFF7
:1033A000F7CF8091E2008E7E80618093E200809171
:1033B000E1008E7E8093E1008091E3028E7E816049
:1033C000E5CF1F920F920FB60F921124CF92DF928A
:1033D000EF92FF920F931F932F933F934F935F931F
:1033E0006F937F938F939F93AF93BF93EF93FF93CD
:1033F000CF93DF93CDB7DEB76C97DEBFCDBF109212
:10340000E9008091E80083FF25C068E0CE01459681
:103410000E94F50C82EF8093E8008D8987FF39C008
:103420009091E80090FFFCCF982F907609F034C17E
:103430009E894F89588D2F89F88C911131C0803821
:1034400061F58091E1028093F1001092F1008EEF1E
:103450008093E8006C960FB6F894DEBF0FBECDBF28
:10346000DF91CF91FF91EF91BF91AF919F918F919C
:103470007F916F915F914F913F912F911F910F918C
:10348000FF90EF90DF90CF900F900FBE0F901F90A6
:1034900018959EEF9093E800C7CF1092F100D5CF1A
:1034A000913059F48111D3CF4130510581F680918B
:1034B000E1028D7F8093E102CACF933049F48111FC
:1034C000C6CF4130510519F68091E1028260F2CFFA
:1034D000953041F48091E80080FFFCCF2068209374
:1034E000E300B5CF963009F0A9C00B8D1C8D22E00A
:1034F0001092E9001092DF021092DE02F2122EC04A
:103500001092DD021092DC020E94C40C1F8299E02E
:103510009983FA8291E09E8390EA98879AEF99873F
:103520002091DE023091DF02275F3F4F3C832B83E7
:103530008D831092E9001092DF021092DE02109348
:10354000DD020093DC0249E050E0BE016F5F7F4F77
:1035500080E00E949E0C0E94C40C79CF1093DD0283
:103560000093DC020E94DB0BDC0112960D911C9192
:103570000115110509F451C1D801ED91FC910480A8
:10358000F581E02DBE016B5E7F4FC8010995009764
:1035900009F03EC1F80100851185EACFF3E0FF1282
:1035A0000EC08F89882309F440C0823061F440E85E
:1035B00060E18DE39FE00E945D1C811148CF81E2B4
:1035C0008093EB0047CF813029F440E86BE081E342
:1035D0009FE0F1CF833099F70E94DB0BDC0112965C
:1035E000ED90FC908E010F5F1F4F6801E114F10414
:1035F00079F0D701ED91FC910680F781E02DB801BB
:10360000C7010995080F111DF701E084F184EECF81
:10361000D8011C92F60101900020E9F73197BF0113
:103620006C197D0940E0C601C6CF6BE17FE0FB016C
:10363000449150E080E80E949E0C09CF973009F435
:10364000BECF983021F481E08093F10000CF993013
:1036500009F0FDCE837009F0B2CFE8E1F1E081E03E
:1036600031E096E32191222371F08093E9003093B9
:10367000EB00DF0111972C912093EC009093ED006B
:103680008F5F873079F78EE78093EA001092EA0027
:103690008F898093F102DBCE8B8D9C8D1092E90097
:1036A0001092DF021092DE029093DD028093DC0222
:1036B000898D811192C08E899D89913A49F4813218
:1036C00009F07DCF47E050E065E071E080E0B3CFE6
:1036D000913209F074CF833269F48F89988DB0E00C
:1036E000A0E08093010190930201A0930301B093A5
:1036F0000401ADCE803269F48091E80082FFFCCFF6
:1037000067E085E091E00E94F50C8BEF8093E80084
:103710009ECE823209F09BCE8F8980930C01EEEF12
:10372000FFE7859194918B3F9C4D51F1E0E0F8E0EB
:103730008091050190910601A0910701B0910801C7
:10374000803B9440A105B105F1F480910C0180FD0E
:103750001AC0EE3F8AE0F80789F587E797E791837B
:103760008083809160008093E00288E19BE00FB647
:10377000F894A895809360000FBE9093600067CE88
:10378000EEEFFAE0D5CF808191818737974709F036
:103790005ECEA895809160008861809360008091E2
:1037A000E00280936000EE3F2AE0F20789F080910A
:1037B000FE0A9091FF0A9183808349CE8081918196
:1037C0008737980751F29093FF0A8093FE0AC5CF7E
:1037D0001092FF0A1092FE0A3ACE0E94DB0BDC0127
:1037E00012960D911C910115110509F4E8CED8012E
:1037F000ED91FC910190F081E02DBE016B5E7F4F59
:10380000C8010995811123CEF80100851185EBCF00
:10381000181619060CF41BCED2CEF1E0FF12BECE64
:103820006FE17FE004CF1F920F920FB60F92112429
:103830002F933F938F939F93AF93BF938091D40225
:103840009091D502A091D602B091D7023091D302C7
:1038500023E0230F2D3758F50196A11DB11D2093AC
:10386000D3028093D4029093D502A093D602B09352
:10387000D7028091D8029091D902A091DA02B0913A
:10388000DB020196A11DB11D8093D8029093D9024D
:10389000A093DA02B093DB02BF91AF919F918F9119
:1038A0003F912F910F900FBE0F901F90189526E813
:1038B000230F0296A11DB11DD2CFEF92FF920F935D
:1038C0001F93CF93DF93F82E192FE62E042F81E05C
:1038D000860F880F0E94700C83E00E94700CCF2D21
:1038E000D12FEC0EFD2EF11CCE15DF05B9F007FF30
:1038F00013C0FE0184910E94700C182F80E00E947A
:10390000700C812321968111EFCFDF91CF911F9110
:103910000F91FF90EF9008958881EDCF81E0F5CF72
:10392000CF93DF931092F5061092F40688EE93E0A1
:10393000A0E0B0E08093F6069093F706A093F80617
:10394000B093F90682E291E09093F3068093F20639
:103950008FEF9FEF9093FF068093FE061092A707CC
:103960001092A6078CE491E09093A5078093A4079A
:1039700010929D0710929C0780E491E090939B0722
:1039800080939A0798E09093A30781E08093A20721
:1039900010929F071092A00710929E078093A10794
:1039A000109293071092920724E331E0309391072D
:1039B000209390079093990780939807109295070A
:1039C000109296071092940780939707C0E6D7E06D
:1039D000198218821B821A821D821C8250E040E0EC
:1039E0006AEF71E0CE010E940C17269687E0C0397D
:1039F000D80771F7C2E4D7E0198218821B821A82B5
:103A00001D821C8250E040E06AEF71E0CE010E940E
:103A10000C17269687E0C036D80771F7DF91CF9153
:103A20000895CF93DF93CDB7DEB760970FB6F894C4
:103A3000DEBF0FBECDBF789484B5826084BD84B5EF
:103A4000816084BD85B5826085BD85B5816085BD99
:103A500080916E00816080936E0010928100809151
:103A600081008260809381008091810081608093D9
:103A7000810080918000816080938000809191001E
:103A80008260809391008091910081608093910089
:103A9000809190008160809390008091C10084604B
:103AA0008093C1008091C10082608093C1008091A9
:103AB000C10081608093C1008091C30081608093C8
:103AC000C3008091C00082608093C0008091C200DA
:103AD00081608093C20080917A00846080937A0034
:103AE00080917A00826080937A0080917A00816070
:103AF00080937A0080917A00806880937A00109297
:103B0000F1021092E1021092E3028091D7008160ED
:103B10008093D70080EA8093D80089B5806189BD01
:103B200089B5826089BD09B400FEFDCF61E070E017
:103B300080E090E00E94270D8091D8008F7C80610A
:103B40008093D8008091E000807F8093E000809196
:103B5000E1008E7E8093E1008DE08093E200559A33
:103B6000209A0E94000F82E48093000180916400FB
:103B70008E7F8093640080917A00806480937A00C5
:103B800080917A0086FDFCCF009178001091790039
:103B90000E94020DAB01BC01C801B0E0A0E0DC0155
:103BA000992788276C017D01C40ED51EE61EF71EDD
:103BB000C701B60120916400216020936400611563
:103BC00071058105910511F00E948F2F1092CF028F
:103BD0001092CE021092D2020E94000F0E94560F45
:103BE00080E80E944B0F8823A9F05C9885EA8EBD7F
:103BF00000000DB407FEFDCF5C9A2E982F982D98EB
:103C00008091640080628093640081E083BF889526
:103C100013BEFCCF84E00E944B0F882309F448C0F8
:103C20002D9884E80E944B0F8823E1F00E94F10E4A
:103C300088EC90E00E94F30E2F9882E090E00E94C2
:103C40002D318F3F29F06FEF82E090E00E943531F7
:103C500084EF91E00E94F30E2F9A84E80E944B0FAC
:103C60008111FBCF84E10E944B0F8823E1F00E9479
:103C7000F10E88EC90E00E94F30E2E9882E090E026
:103C80000E942D31882329F060E082E090E00E94BC
:103C9000353184EF91E00E94F30E2E9A84E10E9468
:103CA0004B0F8111FBCF88EC90E00E94F30EB2CF56
:103CB0000E94F10E82E090E00E94BF15882309F473
:103CC00041C03E9A3F9A81E090E00E94BF1581FF7B
:103CD00013C0082F0470302E82FD2E9801EF1FEFC5
:103CE000B8E0AB2EB12C80E40E944B0F882369F121
:103CF0002E9A2F9A0E94F10E82E390E00E94F30E1A
:103D00000E94F80E8111F8CFE2E04E2E512C612C6A
:103D1000712C8FB7F8944091D4025091D5026091E4
:103D2000D6027091D7028FBF80916402882309F474
:103D3000D0C01092640280E090E0892B51F30E9481
:103D40000000E7CF3E983F98BECF332029F00430E3
:103D5000110511F42E9A2F9881E00E94D607980140
:103D600017FF04C022273327201B310B277033276E
:103D7000C80117FD0796A3E095958795AA95E1F7E9
:103D800017FF05C00197A501421B530B9A01BC0107
:103D90007695762F6627779567956E507D4FF12C37
:103DA000E12C2501421A530A8E3F5FEF950709F473
:103DB0003EC0DB0150E040E0F701E75DF74F4F0107
:103DC0003B01F0E86F0E711C8F3F980781F0F40102
:103DD000E40FF51FE491022E01C0EE0F0A94EAF7FA
:103DE0005496FC915497EF2B5496EC9354972115CD
:103DF0003105B9F0F401E40FF51F24906301C40EFE
:103E0000D51EE22DF0E0042C02C0F595E7950A944A
:103E1000E2F7FE87ED87F6012488FD852F2AF6015B
:103E2000248A4F5F5F4F11964835510569F6019618
:103E3000F8E5EF0EF11C60587F4F40EBE416F104FB
:103E400009F0B2CF0E94560F8FE090E00E94F30E6F
:103E50000F5F1F4F0931110509F045CF332011F0D5
:103E60002F9A2D9880E991E00E94F30E0E94F10EA6
:103E700081E090E00E94BF1580FF3ECF8AE090E095
:103E80000E94BF159FEF980F9E3F08F035CF22E3A9
:103E900030E0309367022093660228E330E03093ED
:103EA0006902209368020BE010E0682F84EA97E033
:103EB0000E94C410C8010E94BF150F5F1F4F01313F
:103EC000110599F70E94560F88EE93E00E94F30EB9
:103ED00013CF80916502942F981B892F9091000138
:103EE000891748F48F5F891708F025CF81E083BFD9
:103EF000889513BE20CF81E08093640240936502D1
:103F00008091620290916302019690936302809384
:103F1000620280916B0280936A020E94F80E809385
:103F20006B028091D2028111F5C02091CE023091B6
:103F3000CF02E2EFF2E081118FEF002481938193B1
:103F4000819381930394D1F71092690210926802D1
:103F500010926702109266021092D1021092D00263
:103F60002130310561F48091CC029091CD024F97C0
:103F700034F087E190E09093CF028093CE0280915D
:103F8000CE029091CF028831910508F0AEC4FC01B9
:103F9000E453F04E0C94AC33E41F2820F720D220D9
:103FA000D22073219C21B5211A22B320A522A5225B
:103FB000A522A522B122DD227A22FC22FC229F2307
:103FC0009F239F239F230C244FE55EE070E060E079
:103FD00090E080E00E94D7094FE55EE070E060E08D
:103FE00082E690E00E94D7098AE290E0909367020F
:103FF000809366028FE090E090936902809368025C
:1040000066E57EE084EA97E00E94A00E81E7809357
:104010009507809394078AE38093960761E57EE095
:1040200080E997E00E94A00E6FE37EE080E697E0D3
:104030000E947D1681E090E09093CB028093CA02AB
:104040001092C9021092C80241E050E060E04DC0F9
:104050000E946E186091C6027091C702CE0101964F
:104060000E94DD16CE0101960E947813CE010196C2
:104070000E94DC1465E37EE080E697E00E947D16F6
:104080006AE27EE086E697E00E947D166FE17EE0C0
:104090008CE697E00E947D166BE17EE082E797E078
:1040A0000E947D168091C6029091C702892B09F06B
:1040B00057C060E17EE088E797E00E947D166BE0E4
:1040C0007EE08EE797E00E947D1686E090E0909378
:1040D000CB028093CA021092C90281E08093C80289
:1040E0004091CA025091CB0261E080E00E94EE0D47
:1040F0002091CA023091CB0200E04091C802609149
:10410000C9028091D0029091D1020E94501181E0A9
:104110008093D202C090CE02D090CF02B8E1CB16ED
:10412000D10408F07CC4F601E856FF4D0C94AC3382
:1041300092249224922492249224922492246E2BEC
:10414000E22AE22AE22AE62AE62AE62AE22AE22A03
:10415000E62A642C642C642C642C642C642CE22AE3
:1041600084E090E0B4CF0E946E1860E07EE0CE0163
:1041700001960E94A516CE0101960E947813CE01E9
:1041800001960E94DC148EEA92E00E949017409102
:10419000CA025091CB026091C8028091C9020E946C
:1041A000EE0DB5CF0E946E188091CE029091CF0295
:1041B00066EF7DE0039711F06BEE7DE0CE01019696
:1041C0000E94A516CE0101960E947813CE01019699
:1041D0000E94DC1486E992E00E9490174091CA0286
:1041E0005091CB026091C8028091C9027FCF0E949A
:1041F0006E1861EE7DE0CE0107960E94A5166091D3
:10420000C6027091C702CE0101960E94DD16BE0162
:104210006F5F7F4FCE0107960E944C16CE0101962C
:104220000E94DC141A8219821C821B821E821D824B
:104230006F8178856115710531F04B855C85CE0104
:1042400001960E940C17CE0101960E947813CE01B0
:1042500001960E94DC1470E6E72E77E0F72E70E0FE
:1042600060E08B010F5F1F4F8091C6029091C702E3
:10427000681779070CF0B801CE0101960E94DD168F
:10428000BE016F5F7F4FC7010E94C115CE0101962D
:104290000E94DC14A6E0EA0EF11CB80105301105FD
:1042A00001F71093CB020093CA0281E08093C90208
:1042B0008093C80245E050E061E00E94EE0D20913D
:1042C000CA023091CB0200E04091C8026091C9025D
:1042D0008091D0029091D1020E945011CE01079698
:1042E0000E94DC1414CF0E946E1866ED7DE0CE01B2
:1042F00001960E94A516CE0101960E947813CE0168
:1043000001960E94DC146BEC7DE080E697E00E9451
:104310007D166EEB7DE086E697E00E947D1682E0DA
:1043200090E09093CB028093CA021092C90210923F
:10433000C80242E050E08ACE0E946E1869EB7DE030
:10434000CE0101960E94A516CE0101960E94781317
:10435000CE0101960E94DC146BEA7DE080E697E0D6
:104360000E947D166CE97DE0D6CF6DE87DE082E4A9
:1043700097E00E947D1662E87DE088E497E00E9465
:104380007D166091940270919502CE0101960E9473
:104390003717BE016F5F7F4F88E497E00E944C168D
:1043A000CE0101960E94DC146CE77DE088E497E082
:1043B0000E9422166BE67DE08EE497E00E947D1657
:1043C0006DE57DE084E597E00E947D1660919202A4
:1043D00070919302CE0101960E943717BE016F5F64
:1043E0007F4F84E597E00E944C16CE0101960E9413
:1043F000DC1484E090E090939102809390021092FC
:104400008F020E94E91282E48093950780939407BB
:1044100087E38093960769E97CE080E997E00E9452
:10442000A00E83E490E00E941B1087E690E00E94BB
:104430001B106DCE0E94402F6B017C0167E87CE071
:1044400082E497E00E947D1660E87CE088E497E0D3
:104450000E947D1687E090E090938E0280938D02FB
:1044600083E090E0909391028093900210928F02EB
:10447000C701B601A30192010E944331672B79F471
:104480006BE77CE088E497E00E94221662E77CE01C
:104490008EE497E00E947D160E94E91238CE6BE60A
:1044A0007CE088E497E00E94221661E67CE08EE4DE
:1044B00097E00E947D16809192029091930203975B
:1044C0009093930280939202181619062CF363E5D9
:1044D0007CE084E597E00E947D1684E090E0909374
:1044E00091028093900287E190E090938E028093F6
:1044F0008D02D2CF6BE47DE082E497E00E947D16CE
:104500006DE37DE088E497E00E947D166BE27DE03C
:104510008EE497E00E947D1667E27DE084E597E0F7
:104520000E947D1684E090E0909391028093900227
:1045300010928F020E94E9120E94D51281E090E051
:1045400090938E0280938D02E2CD0E94E9128091B9
:10455000CE029091CF020A9709F4D9CD0E94D512CC
:10456000D6CD64E571E082E497E00E942D176BE6FA
:1045700071E088E497E00E942D1760E871E08EE416
:1045800097E00E942D1767E971E084E597E00E94AB
:104590002D176EEA71E08AE597E00E942D1785E0FD
:1045A00090E0909391028093900281E080938F023B
:1045B0000E94E9128FE090E0C3CF6AEF71E082E4DD
:1045C00097E00E942D1762EC71E088E497E00E946A
:1045D0002D1761ED71E08EE497E00E942D1783E0C6
:1045E00090E0909391028093900210928F020E942B
:1045F000E91287E190E0A4CF60E27DE0419711F0FD
:104600006AE17DE082E497E00E947D1660918B0272
:1046100070918C02CE0101960E94AE16BE016F5FB2
:104620007F4F82E497E00E944C16CE0101960E94D3
:10463000DC1466E27DE088E497E00E947D1665E286
:104640007DE08EE497E00E947D168091CE029091ED
:10465000CF026BE07DE0419711F065E07DE084E5FD
:1046600097E00E947D1661E17DE08AE597E00E9477
:104670007D1685E090E0909391028093900281E016
:1046800080938F020E94E912E0918B02F0918C02DC
:10469000EE0FFF1FEE0FFF1FEA56FD4F2081318105
:1046A000428153816091460770914707E5E0E69F9C
:1046B000C001E79F900D11246AE070E00F960E9400
:1046C0006D148091CE029091CF024197E9F4209130
:1046D0008702309188024091890250918A026EE2ED
:1046E00070E087E390E00E946D140E94901461E0F6
:1046F0007DE0CE0101960E94A516CE0101960E9492
:104700003A14CE010196ECCD87E380939F07809306
:104710009E078EE28093A007E0918B02F0918C02BD
:10472000EE0FFF1FEE0FFF1FE255FD4F408151813D
:10473000628173818AE997E00E94DF13D6CF66EF2A
:104740007CE08331910559F069EE7CE0843191057C
:1047500031F06BED7CE0459711F06CEC7CE082E48D
:1047600097E00E947D1660E07DE088E497E00E947B
:104770007D166FEF7CE08EE497E00E947D168091BD
:104780008D0290918E026BEB7CE0059711F063EB4C
:104790007CE084E597E00E947D1663EC7CE08AE58E
:1047A00097E00E947D1685E090E0909391028093BF
:1047B000900281E080938F020E94E91280918D0225
:1047C00090918E020597F9F4209183023091840232
:1047D000409185025091860265E270E082E390E0AC
:1047E0000E946D14209187023091880240918902C5
:1047F00050918A026EE270E087E390E00E946D14AF
:104800006FEA7CE076CF20917F0230918002409168
:10481000810250918202E0CF60917F02709180020C
:10482000809181029091820200918702109188020A
:104830002091890230918A02600F711F821F931F9D
:1048400000918302109184022091850230918602AA
:10485000601B710B820B930B0E94103020E030E044
:104860004CEF51E40E944A320E9455330E94F232CA
:104870000E94BC326B016AEF71E082E497E00E9413
:104880002D176FED71E088E497E00E942D176CEE14
:1048900071E08EE497E00E942D17B6016536710530
:1048A00014F064E670E0CE0101960E943717BE0155
:1048B0006F5F7F4F8EE497E00E944C16CE01019609
:1048C0000E94DC146BEF71E084E597E00E942D17E5
:1048D00010928F0284E090E0909391028093900276
:1048E00010928E0210928D02D7CD85E090E09093C9
:1048F000670280936602909369028093680268EA77
:104900007CE084EA97E00E94A00E4091CE02509194
:10491000CF02052E000C660B770B84EA97E00E940D
:10492000DF13F5CB80E80E94400F81111AC080E1AF
:104930000E94400F811115C080E20E94400F81113A
:1049400010C080E40E94400F81110BC088E00E94DB
:10495000400F811106C084E00E94400F882309F4B3
:104960005EC0A090CA02B090CB023090C802E09026
:10497000D002F090D10201E09501432D6091C9026F
:10498000C7010E945011B5010B2C000C880B990B2C
:104990000E94103020E030E040E05FE30E946F3082
:1049A0006D877E878F87988B20E030E0A9010E9479
:1049B0004A3320E030E040E05FE387FD33C06D859F
:1049C0007E858F8598890E94DE310E94BC328B01E2
:1049D00088248394912CE616F7061CF032E0832E8F
:1049E000912C80E10E94400F882359F1EFEFEE1ADD
:1049F000FE0AEA14FB04ECF4F092D102E092D00239
:104A00002091CA023091CB0200E04091C80260912F
:104A1000C9028091D0029091D1020E9450110E944F
:104A2000560F89C96D857E858F8598890E94DD31F5
:104A3000CCCFF1E0AF1AB108B092D102A092D0026F
:104A4000DFCF80E80E94400F882371F001E0E01A78
:104A5000F108F092D102E092D002F7FED1CF10928D
:104A6000D1021092D002CCCF80E40E94400F882364
:104A7000D9F03320A9F08A94892891F4E00EF11E30
:104A8000F092D102E092D0028091D0029091D102B6
:104A90008A159B050CF4B4CF41E0A41AB108CCCF21
:104AA0003FEFE31AF30AECCF80E20E94400F882325
:104AB000B9F0332089F052E08516910469F4E01AC8
:104AC000F10AF092D102E092D0028091D00290914E
:104AD000D10297FF95CFC3CF81E0E81AF108F1CF5B
:104AE00088E00E94400F882309F459C51092D20231
:104AF00093E0C916D10409F4BFC308F05AC0B1E06D
:104B0000CB16D10409F486C0E2E0CE16D10409F434
:104B1000B0C0EF2809F074CF81E090E09093CF020D
:104B20008093CE0220ED37E040E050E020938702F2
:104B3000309388024093890250938A0288E893E177
:104B4000A0E0B0E08093830290938402A09385025A
:104B5000B093860210927F0210928002109281021E
:104B6000109282021092C7021092C60210927E0228
:104B700010927D0284E690E090937C0280937B0209
:104B800082E390E09093930280939202EEEAF2E047
:104B900086EC92E011921192119211928E179F075A
:104BA000C9F71092CD021092CC0280E00E94E4146A
:104BB00027CFF5E0CF16D10409F47EC408F423C44E
:104BC00016E0C116D10409F0A4CF86E090E09093DE
:104BD0008E0280938D0210927702109278021092CA
:104BE000790210927A02E114F10409F4C9C4EA943A
:104BF000EF2809F005CF86E190E09093CF028093F3
:104C0000CE0280917F0290918002A0918102B091AA
:104C1000820221C4D0928E02C0928D0292E0E916E7
:104C2000F104F1F074F4E114F104B9F084E090E0DF
:104C3000EA94EF2809F0E4CE9093CF028093CE025D
:104C4000DFCEE4E0EE16F10489F06CF086E090E04F
:104C500005E0E016F10481F3D3CE83E090E0ECCFE1
:104C600089E090E0E9CF82E090E0E6CF85E090E057
:104C7000E3CF8091C6029091C702E816F9061CF0B6
:104C80001FEFE11AF10AF092C702E092C60281E03A
:104C90000E94E4140E94402F24E130E040E050E004
:104CA0000E9443319B0141E050E050938E024093BB
:104CB0008D0210928F02FB013197E131F10508F06E
:104CC000D6C2EB59F94D0C94AC3376269D26BC2602
:104CD000EF26EF261A271A2747278E278E278E279B
:104CE000F027F02744286528942804296AEC7BE003
:104CF00082E497E00E947D166CEB7BE088E497E00D
:104D00000E947D1663EB7BE08EE497E00E947D16A7
:104D100083E090E0909391028093900222E030E053
:104D200040E050E02093AA023093AB024093AC02E3
:104D30005093AD028AE090E07FCF62EA7BE082E4AC
:104D400097E00E947D1662E97BE088E497E00E948C
:104D50007D1682E090E090939102809390028AE722
:104D600090E0A0E0B0E08093A2029093A302A09311
:104D7000A402B093A502DECF61E87BE082E497E075
:104D80000E947D1663E77BE088E497E00E947D1631
:104D900062E67BE08EE497E00E947D1669E57BE0A9
:104DA00084E597E00E947D1684E090E09093910264
:104DB000809390020E94402F2EE734E040E050E0C4
:104DC0000E9443316E5A7C4F8F4F9F4F60939A02DF
:104DD00070939B0280939C0290939D02ABCF6DE4F5
:104DE0007BE082E497E00E947D166EE37BE088E43E
:104DF00097E00E947D1660E37BE08EE497E00E94DE
:104E00007D1666E27BE084E597E00E947D1684E0F3
:104E100090E090939102809390020E94402F29EAA3
:104E200031E640E050E00E944331605B794B8F4FA8
:104E30009F4FCCCF66E17BE082E497E00E947D1635
:104E400064E07BE088E497E00E947D1661EF7AE001
:104E50008EE497E00E947D1683E090E090939102AB
:104E6000809390020E94402F21E63AEE40E050E00D
:104E70000E9443316058774C8E4F9F4F609396024B
:104E800070939702809398029093990253CF61EEAA
:104E90007AE082E497E00E947D1662ED7AE088E491
:104EA00097E00E947D1682E090E0909391028093BB
:104EB000900260918702709188028091890290919E
:104EC0008A020E94103020E030E040E450E40E946A
:104ED0004A326B017C0120E030E0A9010E944A3394
:104EE00020E030E040E05FE387FD13C0C701B6017A
:104EF0000E94DE310E94BC32660F771F881F991F07
:104F000060938702709388028093890290938A024B
:104F100011CFC701B6010E94DD31ECCFEEEAF2E01D
:104F200046EC52E090E080E0C190D190E190F190A9
:104F30008C0D9D1D4E175F07B9F7C2970CF43FC348
:104F400082E090E02930310539F084E090E02A30A9
:104F5000310511F085E090E09093950280939402E2
:104F600062EC7AE082E497E00E947D166DEB7AE0D5
:104F700088E497E00E947D166091940270919502FA
:104F800061507109CE0101960E943717BE016F5F13
:104F90007F4F88E497E00E944C16CE0101960E9454
:104FA000DC1465EB7AE088E497E00E94221668EA58
:104FB0007AE08EE497E00E947D166DE97AE084E560
:104FC00097E00E947D1684E090E090939102809398
:104FD000900287E090E090938E0280938D02AACE9B
:104FE0008091870290918802A0918902B0918A02F3
:104FF000843F9140A105B1050CF4E1C20E949812D2
:1050000005970CF4DCC20E94402F23E030E040E022
:1050100050E00E9443316B016EE87AE082E497E051
:105020000E947D16F2E0CF16D104C8F465E77AE05D
:10503000CD2811F066E67AE088E497E00E947D16BC
:1050400061E87AE08EE497E00E947D1683E090E0CC
:1050500090939102809390028BE090E0EDCD67E514
:105060007AE088E497E00E947D1667E47AE08EE4B7
:1050700097E00E947D166EE37AE084E597E00E9457
:105080007D1684E090E0E4CF6CE27AE082E497E081
:105090000E947D166BE17AE088E497E00E947D161D
:1050A00069E07AE08EE497E00E947D1666EF79E091
:1050B00084E597E00E947D1684E090E09093910251
:1050C000809390028DE090E0B7CD8091870290911F
:1050D0008802A0918902B0918A028C329140A10588
:1050E000B1050CF46CC263EE79E082E497E00E94B3
:1050F0007D1663ED79E088E497E00E947D1662EC0E
:1051000079E08EE497E00E947D1667EB79E084E514
:1051100097E00E947D1684E090E090939102809346
:1051200090028CE090E088CD0E94981208970CF4D1
:1051300046C20E94402F27E030E040E050E00E944D
:1051400043318B010F5F1F4F0E94402F26E030E05C
:1051500040E050E00E9443316B01FB01EE0FFF1F66
:10516000EE0FFF1FE255FD4FA801012E000C660B4C
:10517000770B80819181A281B381840F951FA61F37
:10518000B71F80839183A283B3836CEA79E082E4C2
:1051900097E00E947D16B801CE0101960E94371754
:1051A000BE016F5F7F4F82E497E00E944C16CE01F4
:1051B00001960E94DC1461EA79E088E497E00E949D
:1051C0007D16B601CE0101960E94AE16BE016F5F3C
:1051D0007F4F88E497E00E944C16CE0101960E9412
:1051E000DC1469E072E08EE497E00E942D176BE119
:1051F00072E084E597E00E942D1784E090E09093A0
:1052000091028093900296CD69E272E082E497E089
:105210000E942D1768E372E088E497E00E942D1742
:105220006AE472E08EE497E00E942D1769E572E06F
:1052300084E597E00E942D1784E090E0909391021E
:10524000809390020E94402F27E232E040E050E03D
:105250000E94433166507F4F8F4F9F4F60939E0255
:1052600070939F028093A0029093A10263CD50930C
:10527000CF024093CE02C4CB0E9498128C01D092F0
:105280008E02C0928D02F0928C02E0928B02181670
:105290001906F4F16DE47CE082E497E00E947D164B
:1052A0006CE47CE088E497E00E947D166CE37CE08F
:1052B0008EE497E00E947D1666E37CE084E597E04B
:1052C0000E947D1660918B0270918C02CE01019636
:1052D0000E94AE16BE016F5F7F4F84E597E00E948B
:1052E0004C16CE0101960E94DC1464E37CE084E558
:1052F00097E00E94221684E090E0909391028093C0
:10530000900210928F028091CE029091CF0263CED4
:10531000F701EE0FFF1FEE0FFF1FEA56FD4FC08093
:10532000D180E280F3806091870270918802809141
:10533000890290918A026C157D058E059F0544F5C2
:105340006EE27CE082E497E00E947D166DE27CE0F4
:1053500088E497E00E947D166CE17CE08EE497E0A3
:105360000E947D1660918B0270918C02CE01019695
:105370000E94AE16BE016F5F7F4F84E597E00E94EA
:10538000C115CE0101960E94DC146AE17CE0AFCF2A
:1053900021E130E03093CF022093CE0210927702C9
:1053A000109278021092790210927A020E941030C4
:1053B0004B015C01C701B6010E9410309B01AC019A
:1053C000C501B4010E944A320E94F2320E94BC32EE
:1053D00060936C0270936D0280936E0290936F02E3
:1053E000012E000C220B330B06171707280739076D
:1053F0000CF006CB00936C0210936D0220936E02AA
:1054000030936F02FDCA84E090E090938E02809307
:105410008D02F0928C02E0928B02F701EE0FFF1FDB
:10542000EE0FFF1FE255FD4F80819181A281B38174
:10543000181619061A061B06BCF422E130E0309358
:10544000CF022093CE02109277021092780210922F
:10545000790210927A0280936C0290936D02A0936D
:105460006E02B0936F02CCCA64E17CE082E497E004
:105470000E947D1663E17CE088E497E00E947D163F
:1054800060E07CE08EE497E00E947D1660918B02E4
:1054900070918C02CE0101960E94AE16BE016F5F24
:1054A0007F4F84E597E00E94C115CE0101960E94CE
:1054B000DC146EEF7BE01BCFD0928E02C0928D0287
:1054C00010927702109278021092790210927A026A
:1054D000E114F10419F1EA94EF2809F091CA8091DE
:1054E00076028823D1F162EF7BE082E497E00E94AC
:1054F0007D1663EE7BE088E497E00E947D166CEDFC
:105500007BE08EE497E00E947D1683E090E090932C
:1055100091028093900210928F020CCC83E190E074
:105520009093CF028093CE024091870250918802DF
:105530006091890270918A02809183029091840225
:10554000A0918502B0918602481759076A077B0728
:105550000CF081CFDB01CA017ECF84E190E0909313
:10556000CF028093CE0228E833E140E050E0209360
:105570006C0230936D0240936E0250936F0240CAEA
:1055800085E190E09093CF028093CE0280918702D4
:1055900090918802A0918902B0918A025CCF84E048
:1055A0000E94400F882309F42BCA42E0C41AD10894
:1055B00055E0C516D10408F023CA1092D20281E04A
:1055C00090E03ACB81E00E94BA1229CA80E00E94A2
:1055D000BA12811124CA88E00E94400F882309F47E
:1055E0001ECA1092D2028091CE029091CF028C30CE
:1055F000910509F44EC060F50B9709F010CA80912F
:105600007D0290917E02019690937E0280937D02AE
:105610008091870290918802A0918902B0918A02BC
:1056200080599140A109B109809387029093880223
:10563000A0938902B0938A0280917B0290917C02B0
:10564000059790937C0280937B0281E090E041C0BB
:105650008D309105E1F1409709F0E1C98091870211
:1056600090918802A0918902B0918A02885E93404D
:10567000A109B1098093870290938802A0938902BF
:10568000B0938A0282E390E0909393028093920217
:10569000DCCF80917B0290917C020A9690937C02F1
:1056A00080937B028091870290918802A091890269
:1056B000B0918A02885C9109A109B109809387029F
:1056C00090938802A0938902B0938A02BECF8EE0A5
:1056D00090E09093CF028093CE02A1C984E00E9413
:1056E000400F882309F440C01092D2020E94402F3C
:1056F000A30192010E944331672B682B692BB9F4F7
:1057000060E979E082E497E00E947D1665E879E03F
:1057100088E497E00E947D1682E090E090939102E9
:105720008093900210928F0281E090E016C065E7AE
:1057300079E082E497E00E947D166FE679E088E4E4
:1057400097E00E947D1682E090E090939102809312
:10575000900210928F0288E090E090938E028093E6
:105760008D028AE090E0B5CF88E00E94400F882348
:1057700009F455C91092D20280917D0290917E0267
:10578000892BE9F460E679E082E497E00E947D16D7
:1057900062E579E088E497E00E947D1665E479E0AF
:1057A0008EE497E00E947D1683E090E09093910252
:1057B0008093900210928F0287E090E0CECF0E94FB
:1057C000402FA30192010E944331672B682B692B64
:1057D00049F464E479E082E497E00E947D1664E392
:1057E00079E0ADCF809194029091950201979093CA
:1057F000950280939402181619064CF463E379E03D
:1058000082E497E00E947D1662E279E098CF0E94E0
:10581000402F23EE34E040E050E00E9443318B0102
:1058200002511D4F60E179E082E497E00E947D160D
:105830006FEF78E088E497E00E947D16B801CE0112
:1058400001960E943717BE016F5F7F4F88E497E093
:105850000E944C16CE0101960E94DC146CEE78E09A
:105860008EE497E00E947D1669ED78E084E597E08C
:105870000E947D1684E090E09093910280939002C4
:1058800081E080938F02012E000C220B330B80915C
:10589000870290918802A0918902B0918A02800FBC
:1058A000911FA21FB31F8093870290938802A09339
:1058B0008902B0938A02803B9440A105B1050CF4A3
:1058C00033CF80E190E049CF80E00E94BA1281118D
:1058D000A6C888E00E94400F882309F439C180914E
:1058E000CE029091CF028331910509F4B7C068F4DC
:1058F0008131910509F479C04297C1F11092D20229
:1059000080918D0290918E02E4CE8531910509F44B
:1059100002C108F4CCC0469789F7409177025091B4
:1059200078026091790270917A0280917F02909161
:105930008002A0918102B0918202841B950BA60B7C
:10594000B70B80937F0290938002A0938102B09363
:1059500082028091870290918802A0918902B09181
:105960008A02840F951FA61FB71F36C080918B0235
:1059700090918C02209177023091780240917902C7
:1059800050917A02880F991F880F991FFC01E255E8
:10599000FD4FC080D180E280F380C21AD30AE40AAE
:1059A000F50AC082D182E282F3828A569D4FDC01E1
:1059B0006D917D918D919C910E949C330091870205
:1059C000109188022091890230918A02DC01CB017A
:1059D000800F911FA21FB31F8093870290938802AC
:1059E000A0938902B0938A0289CF80918B02909113
:1059F0008C02209177023091780240917902509187
:105A00007A02880F991F880F991FFC01E255FD4FFC
:105A1000C080D180E280F380C20ED31EE41EF51E4A
:105A2000C082D182E282F3828A569D4FFC0160815E
:105A30007181828193810E949C3300918702109131
:105A400088022091890230918A0268017901C61A80
:105A5000D70AE80AF90AD701C601BECF40917702FA
:105A6000509178026091790270917A02809183025C
:105A700090918402A0918502B0918602841B950BBF
:105A8000A60BB70B8093830290938402A0938502A8
:105A9000B09386028091870290918802A09189023A
:105AA000B0918A02841B950BA60BB70B95CF409142
:105AB0007702509178026091790270917A02809118
:105AC000830290918402A0918502B0918602840F96
:105AD000951FA61FB71F8093830290938402A09303
:105AE0008502B09386028091870290918802A091EE
:105AF0008902B0918A02840F951FA61FB71F809359
:105B0000870290938802A0938902B0938A0281E071
:105B100080937602F3CE40917702509178026091A3
:105B2000790270917A0280917F0290918002A09117
:105B30008102B0918202840F951FA61FB71F809328
:105B40007F0290938002A0938102B0938202A2CF41
:105B50008FB7F894C090D402D090D502E090D602CE
:105B6000F090D7028FBF8091CE029091CF024197E3
:105B700001E010E0029710F00AE010E0809172025C
:105B800090917302A0917402B0917502B701A601C1
:105B9000481B590B6A0B7B0B80917002909171022C
:105BA000823091050CF0F5C0453F5140610571050B
:105BB00010F40C940F25019690937102809370025B
:105BC00080E80E944B0F8823C1F1C0927202D092EC
:105BD0007302E0927402F092750280916C029091CF
:105BE0006D02A0916E02B0916F02012E000C220B8B
:105BF000330B409177025091780260917902709155
:105C00007A026C017D01C01AD10AE20AF30AC416B5
:105C1000D506E606F7060CF447C0040F151F261F2D
:105C2000371F009377021093780220937902309304
:105C30007A020E9490140C940F2580E40E944B0F6E
:105C4000882309F443C0C0927202D0927302E0929A
:105C50007402F092750240916C0250916D02609155
:105C60006E0270916F022AE0209FC001219F900D6B
:105C70001124092E000CAA0BBB0B00917702109186
:105C800078022091790230917A026A017B01C81A68
:105C9000D90AEA0AFB0AC016D106E206F3066CF03E
:105CA000800F911FA21FB31F8093770290937802F9
:105CB000A0937902B0937A02BCCF409377025093BD
:105CC00078026093790270937A02B3CF80E10E94E8
:105CD0004B0F882339F1C0927202D0927302E09286
:105CE0007402F0927502012E000C220B330B80918E
:105CF000770290917802A0917902B0917A02801790
:105D00009107A207B3072CF0801B910BA20BB30BDA
:105D1000CBCF1092770210927802109279021092F3
:105D20007A0287CF80E20E944B0F882321F1C09234
:105D30007202D0927302E0927402F09275028AE0CD
:105D4000809FA001819F500D1124052E000C660B31
:105D5000770B8091770290917802A0917902B091AF
:105D60007A0284179507A607B7079CF2841B950B48
:105D7000A60BB70B99CF1092720210927302109279
:105D800074021092750210927102109270020C94BB
:105D90000F25453651056105710508F011CF0C94AA
:105DA0000F25CF93DF938AE597E00E94DC1484E50A
:105DB00097E00E94DC148EE497E00E94DC1488E4F3
:105DC00097E00E94DC1482E497E00E94DC14C0E9B2
:105DD000D7E02697CE010E94DC1487E0C036D807B2
:105DE000C1F7DF91CF9108958F929F92AF92BF92AA
:105DF000CF92DF92EF92FF92CF93DF93EC01688115
:105E000079818A819B81611571058105910521F454
:105E100064E279ED8BE597E02DE133EF41E050E06E
:105E20000E94433149015A019B01AC01A7EAB1E448
:105E30000E9462316B017C01ACEEB4EFA5019401CC
:105E40000E947031C60ED71EE81EF91EF7FE06C06E
:105E500081E0C81AD108E10880E8F80AC882D9822E
:105E6000EA82FB82C701B6019F77DF91CF91FF9055
:105E7000EF90DF90CF90BF90AF909F908F9008955C
:105E80008F929F92AF92BF92CF92DF92EF92FF924A
:105E900060910D0170910E0180910F0190911001A0
:105EA000611571058105910521F464E279ED8BE5B9
:105EB00097E02DE133EF41E050E00E94433149018A
:105EC0005A019B01AC01A7EAB1E40E9462316B0167
:105ED0007C01ACEEB4EFA50194010E947031C60EB6
:105EE000D71EE81EF91EF7FE06C081E0C81AD108C9
:105EF000E10880E8F80AC0920D01D0920E01E0920C
:105F00000F01F0921001C701B6019F77FF90EF904B
:105F1000DF90CF90BF90AF909F908F900895609347
:105F20000D0170930E0180930F019093100108955D
:105F3000FB01DC0105900D920020E1F70895FC01C2
:105F400005900020E9F7809590958E0F9F1F08958A
:105F5000BB274A3031F4992322F4BDE29095819514
:105F60009F4F0C94E52FBB272A3051F4992342F41C
:105F7000BDE290958095709561957F4F8F4F9F4FB3
:105F80000C94C32FBB27FA01A62F62177105810558
:105F90009105330B30FB66F0AA27660F771F881F29
:105FA000991FAA1FA21710F0A21B63953850A9F7DA
:105FB000A05DAA3308F0A95DA19336F7B111B193A2
:105FC0001082CA010C94FE2FBB27FB015527AA277C
:105FD000880F991FAA1FA41710F0A41B8395505176
:105FE000B9F7A05DAA3308F0A95DA193009779F7EE
:105FF000B111B1931192CB010C94FE2FDC01FC0185
:10600000672F71917723E1F7329704C07C916D93EC
:1060100070836291AE17BF07C8F30895E89409C072
:1060200097FB3EF490958095709561957F4F8F4FCB
:106030009F4F9923A9F0F92F96E9BB279395F695E1
:10604000879577956795B795F111F8CFFAF4BB0F5F
:1060500011F460FF1BC06F5F7F4F8F4F9F4F16C0C3
:10606000882311F096E911C0772321F09EE8872F4D
:10607000762F05C0662371F096E8862F70E060E009
:106080002AF09A95660F771F881FDAF7880F969582
:10609000879597F90895990F0008550FAA0BE0E826
:1060A000FEEF16161706E807F907C0F012161306DA
:1060B000E407F50798F0621B730B840B950B39F41A
:1060C0000A2661F0232B242B252B21F408950A2680
:1060D00009F4A140A6958FEF811D811D08950E94AE
:1060E00082300C94F3300E94E53038F00E94EC309E
:1060F00020F0952311F00C94DC300C94E230112444
:106100000C9427310E94043170F3959FC1F3950FD1
:1061100050E0551F629FF001729FBB27F00DB11D2B
:10612000639FAA27F00DB11DAA1F649F6627B00DBB
:10613000A11D661F829F2227B00DA11D621F739FA4
:10614000B00DA11D621F839FA00D611D221F749FB2
:106150003327A00D611D231F849F600D211D822FF9
:10616000762F6A2F11249F5750409AF0F1F0882320
:106170004AF0EE0FFF1FBB1F661F771F881F91504D
:106180005040A9F79E3F510580F00C94DC300C94F0
:1061900027315F3FE4F3983ED4F386957795679572
:1061A000B795F795E7959F5FC1F7FE2B880F911D77
:1061B0009695879597F9089597F99F6780E870E01D
:1061C00060E008959FEF80EC089500240A9416166D
:1061D000170618060906089500240A9412161306D5
:1061E000140605060895092E0394000C11F4882363
:1061F00052F0BB0F40F4BF2B11F460FF04C06F5F7F
:106200007F4F8F4F9F4F089557FD9058440F551F54
:1062100059F05F3F71F04795880F97FB991F61F028
:106220009F3F79F087950895121613061406551F9F
:10623000F2CF4695F1DF08C0161617061806991F0B
:10624000F1CF86957105610508940895E894BB2700
:1062500066277727CB0197F90895F999FECF92BD6C
:1062600081BDF89A992780B50895262FF999FECF18
:106270001FBA92BD81BD20BD0FB6F894FA9AF99A63
:106280000FBE01960895052E97FB1EF400940E9400
:106290005A3157FD07D00E94AC3107FC03D04EF4B1
:1062A0000C945A3150954095309521953F4F4F4F62
:1062B0005F4F089590958095709561957F4F8F4FB2
:1062C0009F4F08950E94CE31A59F900DB49F900DD1
:1062D000A49F800D911D11240895B7FF0C94623185
:1062E0000E946231821B930B08952F923F924F922E
:1062F0005F926F927F928F929F92AF92BF92CF9256
:10630000DF92EF92FF920F931F93CF93DF93CDB75E
:10631000DEB7CA1BDB0B0FB6F894DEBF0FBECDBFD6
:1063200009942A88398848885F846E847D848C84A7
:106330009B84AA84B984C884DF80EE80FD800C81B0
:106340001B81AA81B981CE0FD11D0FB6F894DEBF93
:106350000FBECDBFED010895A1E21A2EAA1BBB1BF3
:10636000FD010DC0AA1FBB1FEE1FFF1FA217B30721
:10637000E407F50720F0A21BB30BE40BF50B661F37
:10638000771F881F991F1A9469F7609570958095FB
:1063900090959B01AC01BD01CF010895A29FB00172
:1063A000B39FC001A39F700D811D1124911DB29F49
:1063B000700D811D1124911D08955058BB27AA27E7
:1063C0000E94F5310C94F3300E94E53038F00E94C1
:1063D000EC3020F039F49F3F19F426F40C94E230AD
:1063E0000EF4E095E7FB0C94DC30E92F0E940431B9
:1063F00058F3BA17620773078407950720F079F4FA
:10640000A6F50C9426310EF4E0950B2EBA2FA02D94
:106410000B01B90190010C01CA01A0011124FF2751
:10642000591B99F0593F50F4503E68F11A16F0404C
:10643000A22F232F342F4427585FF3CF469537954B
:106440002795A795F0405395C9F77EF41F16BA0B10
:10645000620B730B840BBAF09150A1F0FF0FBB1FBE
:10646000661F771F881FC2F70EC0BA0F621F731F07
:10647000841F48F4879577956795B795F7959E3F64
:1064800008F0B0CF9395880F08F09927EE0F9795F5
:10649000879508950E945E320C94F3300E94EC3090
:1064A00058F00E94E53040F029F45F3F29F00C9449
:1064B000DC3051110C9427310C94E2300E940431ED
:1064C00068F39923B1F3552391F3951B550BBB2723
:1064D000AA2762177307840738F09F5F5F4F220F68
:1064E000331F441FAA1FA9F335D00E2E3AF0E0E85F
:1064F00032D091505040E695001CCAF72BD0FE2FA9
:1065000029D0660F771F881FBB1F2617370748073C
:10651000AB07B0E809F0BB0B802DBF01FF279358F4
:106520005F4F3AF09E3F510578F00C94DC300C94AC
:1065300027315F3FE4F3983ED4F3869577956795CE
:10654000B795F7959F5FC9F7880F911D9695879529
:1065500097F90895E1E0660F771F881FBB1F621748
:1065600073078407BA0720F0621B730B840BBA0B06
:10657000EE1F88F7E09508950E94C3326894B11128
:106580000C94273108950E940C3188F09F5798F0A1
:10659000B92F9927B751B0F0E1F0660F771F881F28
:1065A000991F1AF0BA95C9F714C0B13091F00E9442
:1065B0002631B1E008950C942631672F782F882773
:1065C000B85F39F0B93FCCF3869577956795B39569
:1065D000D9F73EF490958095709561957F4F8F4FD8
:1065E0009F4F08950E94323390F09F3748F49111E5
:1065F00016F00C94273160E070E080E89FEB08957E
:1066000026F41B16611D711D811D0C9409330C9419
:106610002433882371F4772321F09850872B762F29
:1066200007C0662311F499270DC09051862B70E0A6
:1066300060E02AF09A95660F771F881FDAF7880FB7
:106640009695879597F908959F3F31F0915020F4E2
:10665000879577956795B795880F911D969587953E
:1066600097F908950E940C31A0F0BEE7B91788F49D
:10667000BB279F3860F41616B11D672F782F882727
:10668000985FF7CF869577956795B11D9395963965
:10669000C8F308950E944B3008F48FEF089519F461
:1066A00016F40C94E2300C9424330E940C31B8F3AD
:1066B0009923C9F3B6F39F57550B87FF0E94953373
:1066C0000024A0E640EA900180585695979528F45A
:1066D000805C660F771F881F20F026173707480752
:1066E00030F4621B730B840B202931294A2BA695A9
:1066F00017940794202531254A2758F7660F771FEE
:10670000881F20F026173707480730F4620B730BF9
:10671000840B200D311D411DA09581F7B901842FF7
:106720009158880F96958795089591505040660F1F
:10673000771F881FD2F70895DB018F939F930E94E4
:106740006231BF91AF91A29F800D911DA39F900DCB
:10675000B29F900D11240895EE0FFF1F0590F49144
:10676000E02D09940F931F93CF93DF93823091050F
:1067700010F482E090E0E091AA07F091AB0730E0DE
:1067800020E0B0E0A0E0309799F42115310509F43C
:106790004AC0281B390B24303105D8F58A819B81EA
:1067A0006115710589F1FB0193838283FE0111C09C
:1067B000408151810281138148175907E0F0481741
:1067C000590799F4109761F012960C93129713964B
:1067D0001C933296CF01DF91CF911F910F910895B5
:1067E0000093AA071093AB07F4CF2115310551F0A0
:1067F0004217530738F0A901DB019A01BD01DF01FF
:10680000F801C1CFEF01F9CF9093AB078093AA07AE
:10681000CDCFFE01E20FF31F8193919322503109F6
:1068200039832883D7CF2091A8073091A907232B3C
:1068300041F420911301309114013093A907209362
:10684000A80720911101309112012115310541F461
:106850002DB73EB74091150150911601241B350B01
:10686000E091A807F091A907E217F307A0F42E1B07
:106870003F0B2817390778F0AC014E5F5F4F2417A4
:10688000350748F04E0F5F1F5093A9074093A807A4
:10689000819391939FCFF0E0E0E09CCFCF93DF9383
:1068A0000097E9F0FC01329713821282A091AA07A7
:1068B000B091AB07ED0130E020E01097A1F420810A
:1068C0003181820F931F2091A8073091A9072817C3
:1068D000390709F061C0F093A907E093A807DF9199
:1068E000CF910895EA01CE17DF07E8F54A815B8171
:1068F0009E0141155105B1F7E901FB83EA834991F6
:106900005991C40FD51FEC17FD0761F48081918167
:106910000296840F951FE901998388838281938170
:106920009B838A83F0E0E0E012968D919C9113970F
:106930000097B9F52D913C911197CD010296820FE8
:10694000931F2091A8073091A9072817390739F616
:10695000309751F51092AB071092AA07B093A90790
:10696000A093A807BCCFD383C28340815181840FF9
:10697000951FC817D90761F44E5F5F4F88819981D1
:10698000480F591F518340838A819B81938382835F
:106990002115310509F0B0CFF093AB07E093AA07BA
:1069A0009ECFFD01DC01C0CF13821282D7CFB0E0B1
:1069B000A0E0EDEDF4E30C9477318C01009751F4F5
:1069C000CB010E94B2338C01C801CDB7DEB7E0E144
:1069D0000C949331FC01E60FF71F9C012250310902
:1069E000E217F30708F49DC0D901CD91DC9111970E
:1069F000C617D70798F0C530D10530F3CE010497FC
:106A00008617970708F3C61BD70B2297C193D1931C
:106A10006D937C93CF010E944E34D6CF5B01AC1AAC
:106A2000BD0A4C018C0E9D1EA091AA07B091AB0728
:106A3000512C412CF12CE12C109731F58091A807B5
:106A40009091A9078815990509F05CC0461657066C
:106A500008F058C08091110190911201009741F403
:106A60008DB79EB74091150150911601841B950B6F
:106A7000E817F90708F055C0F093A907E093A807B5
:106A8000F90171836083A0CF8D919C91119712962B
:106A90006C90129713967C901397A815B90559F529
:106AA0006C0142E0C40ED11CCA14DB0420F1AC011D
:106AB0004A195B09DA011296159780F06282738297
:106AC00051834083D9016D937C93E114F10471F0FB
:106AD000D7011396FC93EE93129776CF22968C0FE4
:106AE0009D1FF90191838083F301EFCFF093AB07F2
:106AF000E093AA0769CF4816590608F42C017D01D6
:106B0000D3019ACFCB010E94B2337C01009749F0A8
:106B1000AE01B8010E949435C8010E944E3487012D
:106B200053CF10E000E050CFFB01DC0102C0019028
:106B30000D9241505040D8F70895FB01DC010190BF
:106B40000D920020E1F7089517E0CBEAD7E004C0EA
:106B5000FE010E94AC332196CC3AD107C9F7F894D4
:026B6000FFCF65
:106B620010FFFFFFFF00E100000000000001000035
:106B7200000000AC07800000C1808100000000001E
:106B82000000EF0B5A0D100C050C560C140C320CB5
:106B9200000000004A12C40E8313DF0D0000000043
:106BA200FC11C40E8313DF0D00000000C410C40EDC
:106BB2008313DF0D596F752068616C6C7563696EA4
:106BC200617465206F6E207468650077696C646516
:106BD20073742074726970206F6620796F75720009
:106BE2006C6966652C207374756D626C65206F6EBE
:106BF200746F2074686500737562776179207472AE
:106C020061636B732C20616E64206765740063722C
:106C120065616D6564206279206120747261696EBC
:106C22002E002020204A75737420736179206E6FC4
:106C32000020202020746F2064727567732E00205C
:106C42002047616D65206F76657221002020596FA3
:106C520075722073636F72653A200020206F75741D
:106C6200206F66203130302E006F6E206120646507
:106C72006164206475646520696E007468652073C0
:106C8200756277617921212100546865206D6172F6
:106C92006B657420686173006265656E20666C6F57
:106CA2006F64656420776974680063686561702049
:106CB200686F6D656D61646500616369642121219E
:026CC2002100AF
:00000001FF
